:100000000C942F040C944C040C944C040C94E7288E
:100010000C9405320C944C040C944C040C944C0439
:100020000C944C040C944C040C944C040C94A616A4
:100030000C944C040C944C040C944C040C944C0400
:100040000C94CA180C944C040C94CC140C948E147C
:100050000C944C040C944C040C944C040C944C04E0
:100060000C944C040C944C04A70B6D0D6D0DB10B4E
:10007000BE0BCB0BD80B6D0DDC0B6D0DEA0B6D0DB4
:10008000F40BFE0B2F0C6D0D6D0D6D0D080C150C8A
:10009000220C181229125C122912601273126612B5
:1000A0006C123C224222452248224D2257226122D4
:1000B000F022F022F0226B226D2276227F2289220A
:1000C000F022F022F022F022F02293229F22AF228F
:1000D000B922BC22C522CE22D422F022F022F02264
:1000E000F022F022F022F022F022F022F022F02280
:1000F000F022DD220A2D0D2D122D152D182D1B2D70
:100100001E2D212D242D272D2A2D362D362D362D31
:10011000362D362D362D362D362D302D2D2D332DD9
:10012000084AD73B3BCE016E84BCBFFDC12F3D6C5E
:1001300074319ABD56833DDA3D00C77F11BED9E4C4
:10014000BB4C3E916BAAAABE000000803F05A84CA4
:10015000CDB2D44EB93836A9020C50B99186880870
:100160003CA6AAAA2ABE000000803F003E0D0A005D
:100170006F66663A006F6E3A002C6C617365722090
:10018000002C52583A002C4275663A002C533A0023
:100190002C002C57506F733A002C002C4D506F736D
:1001A0003A003C436865636B003C416C61726D00D2
:1001B0003C486F6D65003C486F6C64003C52756E46
:1001C000003C5175657565003C49646C65005D0DCA
:1001D0000A005B302E39672E363934666232363A81
:1001E000000D0A003D00244E005D0D0A0020530062
:1001F000204600205400204D3800204D3900204D6D
:100200003500204D3400204D3300204D3200204D6C
:100210003100204D30002047393400204739330069
:100220002047393100204739300020473230002044
:10023000473231002047313900204731380020470C
:100240003137002047005B473830005B4733005BA5
:100250004732005B4731005B4730005D0D0A005BB1
:10026000544C4F3A005D0D0A002C005B4739323A7E
:10027000005D0D0A002C003A003330003238005B7C
:1002800047005D0D0A002C005B5052423A00290DD8
:100290000A00206D61782074726176656C2C206D87
:1002A0006D0020616363656C2C206D6D2F73656339
:1002B0005E3200206D617820726174652C206D6D56
:1002C0002F6D696E002C20737465702F6D6D007A30
:1002D00000790078002028003D0024002028747553
:1002E000726E204C61736572206D6F6465206F6E55
:1002F0002C20626F6F6C290D0A002434303D0020E1
:1003000028686F6D696E672070756C6C2D6F6666FE
:100310002C206D6D290D0A002028686F6D696E67AD
:10032000206465626F756E63652C206D736563294B
:100330000D0A2432373D002028686F6D696E6720F2
:100340007365656B2C206D6D2F6D696E290D0A2408
:1003500032363D002028686F6D696E6720666565DE
:10036000642C206D6D2F6D696E290D0A2432353D88
:1003700000290D0A2432343D002028686F6D696E13
:10038000672064697220696E76657274206D61738E
:100390006B3A002028686F6D696E67206379636C23
:1003A000652C20626F6F6C290D0A2432333D0020CA
:1003B0002868617264206C696D6974732C20626FA7
:1003C0006F6C290D0A2432323D002028736F667449
:1003D000206C696D6974732C20626F6F6C290D0A33
:1003E0002432313D0020286175746F20737461726E
:1003F000742C20626F6F6C290D0A2432303D00206E
:10040000287265706F727420696E636865732C2042
:10041000626F6F6C290D0A2431343D00202861720F
:100420006320746F6C6572616E63652C206D6D293D
:100430000D0A2431333D0020286A756E6374696F9C
:100440006E20646576696174696F6E2C206D6D290C
:100450000D0A2431323D00290D0A2431313D00209E
:1004600028737461747573207265706F7274206D77
:1004700061736B3A00202870726F62652070696E3C
:1004800020696E766572742C20626F6F6C290D0A7C
:100490002431303D0020286C696D69742070696ECC
:1004A0007320696E766572742C20626F6F6C290DF3
:1004B0000A24363D0020287374657020656E6162E1
:1004C0006C6520696E766572742C20626F6F6C2982
:1004D0000D0A24353D00290D0A24343D00202864EE
:1004E000697220706F727420696E76657274206D07
:1004F00061736B3A00290D0A24333D002028737480
:10050000657020706F727420696E76657274206DEC
:1005100061736B3A002028737465702069646C65A0
:100520002064656C61792C206D736563290D0A2444
:10053000323D002028737465702070756C73652CD3
:100540002075736563290D0A24313D0024303D0078
:100550002424202876696577204772626C207365B1
:100560007474696E6773290D0A24232028766965DF
:1005700077202320706172616D6574657273290D37
:100580000A24472028766965772070617273657246
:10059000207374617465290D0A24492028766965E1
:1005A00077206275696C6420696E666F290D0A2474
:1005B0004E20287669657720737461727475702097
:1005C000626C6F636B73290D0A24783D76616C75DC
:1005D00065202873617665204772626C20736574AC
:1005E00074696E67290D0A244E783D6C696E65202A
:1005F0002873617665207374617274757020626C03
:100600006F636B290D0A24432028636865636B20A0
:1006100067636F6465206D6F6465290D0A24582037
:10062000286B696C6C20616C61726D206C6F636B00
:10063000290D0A2448202872756E20686F6D696E36
:1006400067206379636C65290D0A7E2028637963CE
:100650006C65207374617274290D0A212028666507
:10066000656420686F6C64290D0A3F2028637572E9
:1006700072656E7420737461747573290D0A6374E6
:10068000726C2D7820287265736574204772626CD5
:10069000290D0A000D0A4772626C20302E39675FFF
:1006A00036393466623236205B27242720666F7223
:1006B0002068656C705D0D0A005D0D0A0044697369
:1006C00061626C656400456E61626C6564004361E3
:1006D0007574696F6E3A20556E6C6F636B6564005C
:1006E000272448277C2724582720746F20756E6C98
:1006F0006F636B00526573657420746F20636F6E57
:1007000074696E7565005B000D0A0050726F62655A
:10071000206661696C0041626F7274206475726951
:100720006E67206379636C6500486172642F736F34
:100730006674206C696D697400414C41524D3A20D9
:10074000000D0A00496E76616C69642067636F640E
:10075000652049443A00556E646566696E6564209B
:1007600066656564207261746500556E737570709E
:100770006F7274656420636F6D6D616E64004D6FA0
:1007800064616C2067726F75702076696F6C61743C
:10079000696F6E004C696E65206F766572666C6F6E
:1007A0007700486F6D696E67206E6F7420656E61AB
:1007B000626C656400416C61726D206C6F636B00EC
:1007C0004E6F742069646C6500454550524F4D2052
:1007D00072656164206661696C2E205573696E676D
:1007E0002064656661756C74730056616C75652074
:1007F0003C203320757365630053657474696E67BC
:100800002064697361626C65640056616C75652073
:100810003C203000496E76616C69642073746174A9
:10082000656D656E7400426164206E756D626572FF
:1008300020666F726D6174004578706563746564DD
:1008400020636F6D6D616E64206C657474657200F9
:100850006572726F723A20006F6B0D0A00001124EE
:100860001FBECFEFD8E0DEBFCDBF11E0A0E0B1E00A
:10087000E0E0F0E702C005900D92A630B107D9F78D
:1008800017E0A6E0B1E001C01D92A333B107E1F784
:100890000E944E040C94FE370C9400000E945C14DD
:1008A0000E94FC220E9448190E94F4318EE1E1E985
:1008B000F5E0DF011D928A95E9F781E080939105CB
:1008C00078949091210794FD80939205C1E00E9455
:1008D00022150E9465090E949D130E9434140E94F3
:1008E000CC280E94C72C0E9464240E941C190E94DC
:1008F0009C270E9477091092910510929305809190
:10090000210781FF03C0C093A10502C01092A10579
:100910000E94D115DCCF6F927F928F929F92AF92FF
:10092000BF92CF92DF92EF92FF920F931F93CF93DC
:10093000DF9300D000D0CDB7DEB73C01D22E470107
:1009400058018091210785FF0BC0C30149835A8359
:100950006B837C830E94212B7C816B815A8149812E
:1009600080919205823031F149835A836B837C8375
:100970000E9427158091910581111CC00E94B3240B
:1009800049815A816B817C81882339F00E94C4158A
:1009900049815A816B817C81E7CF850174012D2DBE
:1009A000C3010E94BB2480919205811103C088E09D
:1009B000809392050F900F900F900F90DF91CF9141
:1009C0001F910F91FF90EF90DF90CF90BF90AF906D
:1009D0009F908F907F906F9008952F923F924F92AB
:1009E0005F926F927F928F929F92AF92BF92CF92BF
:1009F000DF92EF92FF920F931F93CF93DF93CDB7C8
:100A0000DEB7E7970FB6F894DEBF0FBECDBF9A8B67
:100A1000898B1B013A0109871A872B873C87CB8A70
:100A2000DC8AED8AFE8AA98E24E0829E20011124B0
:100A3000840D951D9B8F8A8FCA01840D951D9D8FF6
:100A40008C8FDC018D909D90AD90BC90EA8DFB8DDC
:100A50002081318142815381C501B4010E94AC33B0
:100A60006E8F7F8F88A399A32D960FAD2D97F4E0FD
:100A70000F9F8001112429893A89200F311F3BA340
:100A80002AA3C301800F911F9DA38CA3DC01CD90ED
:100A9000DD90ED90FC90F9012081318142815381FC
:100AA000C701B6010E94AC336EA37FA388A799A7A4
:100AB000D501C401B0588D839E83AF83B887D70119
:100AC000C601B05889839A83AB83BC83F101E40DDE
:100AD000F51D2E8D3F8D48A159A1608171818281C4
:100AE00093810E94AB336B017C01F101E00FF11F98
:100AF0002EA13FA148A559A5608171818281938172
:100B00000E94AB334B015C01A70196016D817E8190
:100B10008F8198850E94C3362B013C01A501940169
:100B200069817A818B819C810E94C3369B01AC01D3
:100B3000C301B2010E94AC332B013C01A501940119
:100B40006D817E818F8198850E94C3364B015C0147
:100B5000A701960169817A818B819C810E94C336AD
:100B60009B01AC01C501B4010E94AB33A30192010A
:100B70000E941F346B017C018091AF0520E030E0C2
:100B8000A901823079F4C701B6010E94883687FD39
:100B900019C02BED3FE049EC50E4C701B6010E94BB
:100BA000AB330EC0C701B6010E948534181654F04D
:100BB0002BED3FE049EC50E4C701B6010E94AC3395
:100BC0006B017C0180901D0790901E07A0901F076D
:100BD000B090200729853A854B855C85CA01B9010B
:100BE0000E94AC33A50194010E94AB339B01AC0180
:100BF000C501B4010E94C3360E9450374B015C010D
:100C000020E030E040E05FE3C701B6010E94C33658
:100C100029853A854B855C850E94C3369F77A5015F
:100C200094010E948C340E9462350E94F9347BA7A3
:100C30006AA7DB01AB2B09F493C14B01A12CB12CAA
:100C4000B98DBB2381F0C501B4010E9425359B01FC
:100C5000AC016B897C898D899E890E94C3366B8B20
:100C60007C8B8D8B9E8BC501B4010E9425354B0179
:100C70005C019B01AC01C701B6010E948C342B01C1
:100C80003C012E968FAD2E97E4E08E9FC00111247B
:100C900029893A89280F391F388F2F8BF101E80FE6
:100CA000F91FD9012D913D914D915C916081718128
:100CB000828193810E94AB33A50194010E948C3400
:100CC0006CAB7DAB8EAB9FABA3019201C301B201B4
:100CD0000E94C3369B01AC0160E070E080E090E4CC
:100CE0000E94AB336B017C012BEA3AEA4AE25EE3F5
:100CF000C301B2010E94C3364B015C0120E030E029
:100D000040E850E4C701B6010E94AC339B01AC013E
:100D1000C501B4010E94C3366CA77DA78EA79FA70B
:100D200020E030E040E05FE3C701B6010E94C33637
:100D300068AB79AB8AAB9BAB1D86E1E0F0E0FA874C
:100D4000E98729853A858AA59BA52817390709F4DB
:100D500007C1FD85FC3008F04AC028A939A94AA975
:100D60005BA969817A818B819C810E94C3366B016A
:100D70007C012CA53DA54EA55FA56D817E818F814F
:100D800098850E94C336A70196010E94AC33B62E07
:100D9000A72E982E892E28A939A94AA95BA96D8169
:100DA0007E818F8198850E94C3366B017C012CA5C2
:100DB0003DA54EA55FA569817A818B819C810E94AA
:100DC000C3369B01AC01C701B6010E94AB336D83F2
:100DD0007E838F8398872D852F5F2D878B2D9A2D6E
:100DE000A92DB82D89839A83AB83BC836BC0A98559
:100DF000BA85BD0180E090E00E942535A3019201F3
:100E00000E94C3366B017C010E94893469837A8316
:100E10008B839C83C701B6010E9446374B015C015E
:100E2000EC8DFD8DC080D180E280F380F7FAF094E4
:100E3000F7F8F094ACA1BDA18D919D910D90BC915E
:100E4000A02D8D879E87AF87B88B29813A814B81F2
:100E50005C81C701B6010E94C3366D837E838F8398
:100E60009887A50194016D857E858F8598890E945C
:100E7000C3369B01AC016D817E818F8198850E9474
:100E8000AC336D837E838F839887A5019401C7015E
:100E9000B6010E94C3366B017C0129813A814B81E6
:100EA0005C816D857E858F8598890E94C3369B0104
:100EB000AC01C701B6010E94AB3369837A838B838F
:100EC0009C831D862D813E814F8158856E8D7F8D3F
:100ED00088A199A10E94AC33EA8DFB8D6083718358
:100EE0008283938329813A814B815C816EA17FA1AA
:100EF00088A599A50E94AC33AAA1BBA16D937D934F
:100F00008D939C9313972CA93DA94EA95FA9EF89B6
:100F1000F88D60817181828193810E94AC33AF89A9
:100F2000B88D6D937D938D939C9313976396CFACFF
:100F300063976296ECACFDAC0EAD1FAD6297298D48
:100F40004B895C896D897E8989899A890E948B0485
:100F500080919105811115C0E985FA853196EFCE12
:100F60006396CFAC63976296ECACFDAC0EAD1FAD53
:100F70006297298D4B895C896D897E89C1010E94A8
:100F80008B04E7960FB6F894DEBF0FBECDBFDF919E
:100F9000CF911F910F91FF90EF90DF90CF90BF9076
:100FA000AF909F908F907F906F905F904F903F9009
:100FB0002F9008958F929F92AF92BF92CF92DF921F
:100FC000EF92FF924B015C0180919205823009F40F
:100FD00047C020E030E040EA51E4C501B4010E947E
:100FE000C3360E9462350E94F9346B017C010E9475
:100FF000411620E030E04AE754E4C501B4010E9404
:10100000C3364B015C0182E38C9DB0018D9D700D58
:10101000112480E090E00E9425359B01AC01C501C0
:10102000B4010E94AB330E9462350E94F934CB01B7
:101030000E949028C114D10499F00E94271521E044
:10104000C21AD1088091910581110AC08FEF90E7F3
:1010500022E0815090402040E1F700C00000EACF3C
:10106000FF90EF90DF90CF90BF90AF909F908F90C8
:1010700008952F923F925F926F927F928F929F92EC
:10108000AF92BF92CF92DF92EF92FF920F931F9396
:10109000CF93DF9300D000D0CDB7DEB7782ED92E16
:1010A0004A015B01622E80919205823009F4AAC048
:1010B0000E9441165090A1050E94D52C882351F022
:1010C0009FB7F894809193058064809393059FBFA8
:1010D0000E94271580919105811194C0C12CE12CAB
:1010E000F12C8701262DB501A401872D9D2D0E948D
:1010F0008B0481E08093A2059FB7F89480919305BB
:101100008260809393059FBF0E942715809191056F
:10111000811178C080919205877FB1F78091A205F7
:10112000813041F49FB7F894809193058064809357
:1011300093059FBF0E94271580919105811162C080
:101140000E941C190E9464240E949C2703EA15E057
:1011500084EEE82E86E0F82E272C3D2CF8016191D4
:101160007191819191918F01F7012191319141917B
:1011700051917F0129833A834B835C830E942735F9
:1011800029813A814B815C810E948C34F101619309
:101190007193819391931F01F5E00F3A1F07F1F6C8
:1011A000C12CE12CF12C8701262DB501A401872D3E
:1011B0009D2D0E948B049FB7F894809193058260C7
:1011C000809393059FBF0E944116809191058111E4
:1011D00019C05092A1050F900F900F900F90DF91C2
:1011E000CF911F910F91FF90EF90DF90CF90BF9024
:1011F000AF909F908F907F906F905F903F902F90D7
:101200000C94282F0F900F900F900F90DF91CF919B
:101210001F910F91FF90EF90DF90CF90BF90AF9014
:101220009F908F907F906F905F903F902F90089548
:101230008091930584FD1AC09FB7F894809193051F
:101240008061809393059FBF0E9494130E94321483
:1012500080919205847351F09FB7F8948091930523
:101260008062809393059FBF0C947B16089583B191
:1012700086719091210796FD02C096E18927882307
:1012800059F00E9418099FB7F894809193058066E1
:10129000809393059FBF089584E0809392050E94F8
:1012A00094130E94C12883E00E941B290E942715E5
:1012B00080919105811108C00E94770910929205D2
:1012C0000E947B160C94CC2808958BE3EFEAF5E09E
:1012D000DF011D928A95E9F76EEC75E080E00E94CF
:1012E0009C21811103C087E00C94F42C0895CF92C7
:1012F000DF92EF92FF920F931F93CF93DF9300D073
:1013000000D0CDB7DEB785E9C82E85E0D82E94EEA3
:10131000E92E96E0F92E02EC15E0F601619171914B
:10132000819191916F01F7012191319141915191F9
:101330007F0129833A834B835C830E94273529816F
:101340003A814B815C810E948C34F80161937193E6
:10135000819391938F01F1EACF16F5E0DF06E9F66C
:101360000F900F900F900F90DF91CF911F910F91E1
:10137000FF90EF90DF90CF9008952F923F924F9281
:101380005F926F927F928F929F92AF92BF92CF9215
:10139000DF92EF92FF920F931F93CF93DF93CDB71E
:1013A000DEB7AB970FB6F894DEBF0FBECDBF98A3E4
:1013B0008F8F8AE3EAEEF5E0DF011D928A95E9F767
:1013C0008AE0EFEAF5E0ACEEB5E001900D928A9587
:1013D000E1F71D8E212C312CA12CB12C19A2512CFE
:1013E0001E8E66246394712C05E0402E99249394FC
:1013F00082E0882E8D8DEF8DF8A1E80FF11D008120
:10140000002309F456C29FEB900F9A3128F00E94F6
:10141000941381E00C946A138F5F8D8FAE01475E49
:101420005F4FBE01635E7F4F8F8D98A10E94DE27C4
:10143000811105C00E94941382E00C946A13C98C38
:10144000DA8CEB8CFC8CC701B6010E9491370E94AC
:10145000F934162F70E080E090E00E9427359B0160
:10146000AC01C701B6010E94AB3320E030E048EC8C
:1014700052E40E94C3360E9426370E94F934073492
:1014800021F00D3409F414C151C1163209F487C09A
:10149000B8F4143158F4113108F0B3C0143009F421
:1014A00050C008F47CC01A3069F117C31C3151F1E7
:1014B00020F4163108F4C5C010C31E3119F10DC354
:1014C000103509F497C098F4153309F457C038F46F
:1014D0001B3209F4BFC0113309F4BCC0FEC21C3377
:1014E00008F0FBC216531093F20587E0C8C01C3504
:1014F00049F020F41A3508F092C0EFC21F3508F405
:1015000097C0EBC261110AC0BE8DBB2329F00E94B7
:10151000941388E10C946A13E1E0EE8F1C31A1F082
:1015200040F4143071F01A3009F0A8C08092EB0535
:10153000A5C0153319F11C3529F11E3109F09EC0E3
:1015400010C09092EB059AC0662339F06A3009F01A
:10155000C4C224E02093EB0508C0F3E0F093EB0550
:1015600004C0611104C04092EB0580E08FC06A3076
:1015700009F0B3C236E03093EB05F7CF87E08093F4
:10158000EB057CC0662339F06A3009F0A6C2A9E0F9
:10159000A093EB05EACF98E09093EB05E6CFBE8DE4
:1015A000B111B5CFE2E0EE8F1230B1F048F4112363
:1015B00081F0113011F51093EC051093EA051FC06E
:1015C000163281F01035B1F01330B9F41093EC05F8
:1015D00006C01092EC0503C0FE8DF093EC059092CE
:1015E000EA050DC0643109F078C224E02093EC05CF
:1015F00081E04CC04092EC0502C01092EA0581E007
:101600003EC0123129F0133131F01092F00505C0BF
:101610009092F00502C08092F00582E030C01A3549
:1016200019F41092EF0502C09092EF0583E027C0F5
:101630001D3519F49092ED0502C01092ED0584E07D
:101640001EC0143119F49092EE0502C01092EE05FE
:1016500085E015C03E8D31115ACF113331F410920F
:10166000F10586E093E09E8F11C06A3009F035C223
:101670009092F10586E0A3E0AE8F08C080E066237B
:1016800029F00E94941387E10C946A13F30102C0BD
:10169000EE0FFF1F8A95E2F7CF019F012A213B2120
:1016A000232B09F440C00E94941385E10C946A1323
:1016B0006111E7CF163018F4133048F014C0183019
:1016C00008F40BC21A30E8F01E3151F006C2123095
:1016D00039F01E3129F011111DC09092F3051AC086
:1016E0008092F30517C0143029F0153031F0909234
:1016F000F50505C08092F50502C01092F50589E058
:101700000AC0193019F08092F40502C01092F40555
:101710008AE001C088E0930102C0220F331F8A953E
:10172000E2F7C901BBCFA82AB92A64CE802F992736
:1017300087FD9095A92FB92FFC01E654F109E531F9
:10174000F10508F0CAC1EC5CFF4F0C94E937C09278
:10175000F605D092F705E092F805F092F90580E0E1
:101760007FC0C092FA05D092FB05E092FC05F09292
:10177000FD0539A1316039A381E072C0C092FE0538
:10178000D092FF05E0920006F092010689A18260E6
:1017900089A382E065C0C0920206D0920306E0925F
:1017A0000406F092050699A1946099A383E058C0BD
:1017B0001093060684E054C0C701B6010E94F434B9
:1017C00060930706709308068093090690930A06B3
:1017D00085E046C0C0920B06D0920C06E0920D0642
:1017E000F0920E0686E03CC0C0920F06D092100622
:1017F000E0921106F092120687E032C0C092130602
:10180000D0921406E0921506F092160688E028C0E1
:10181000C0921806D0921906E0921A06F0921B06A2
:10182000A52DA1605A2E8AE01BC0C0921C06D09242
:101830001D06E0921E06F0921F06B52DB2605B2ECB
:101840008BE00EC0C0922006D0922106E0922206C4
:10185000F0922306E52DE4605E2E8CE001C089E065
:101860008301082E02C0000F111F0A94E2F79801AD
:1018700022213321232B21F00E94941389E12AC7CE
:1018800021E633E002C0359527958A95E2F720FFDF
:101890000DC020E030E0A901C701B6010E948534E7
:1018A00087FF04C00E94941384E014C7202A312AC1
:1018B000A1CD552029F03E8D311102C082E08E8FDE
:1018C00025FE11C08091070690910806A091090697
:1018D000B0910A0680389649A849B10524F00E94C3
:1018E00094138BE1F7C68091ED05813031F4FE8DC4
:1018F000F230A1F520FC32C09DC28091B00581116B
:101900002DC020FE1BC08091EE05813039F523E308
:1019100033E34BEC51E46091F6057091F70580914B
:10192000F8059091F9050E94C3366093F60570930F
:10193000F7058093F8059093F90510C08091BD05D7
:101940009091BE05A091BF05B091C0058093F605AA
:101950009093F705A093F805B093F90530FC10C0FB
:101960008091B9059091BA05A091BB05B091BC05D5
:101970008093130690931406A0931506B093160651
:101980008091EB05813041F426FC04C00E94941341
:101990008CE1A0C6E89426F88091F005882341F0F8
:1019A000813061F019A682E088A791E09FA30BC067
:1019B00022E029A731E038A71FA205C0A1E0A9A70E
:1019C00018A6B2E0BFA38091EE05813021F0EE8D24
:1019D000E330B1F52AC0B8E1EB2EB6E0FB2E00E013
:1019E00010E0C52CD12CC601002E02C0959587951C
:1019F0000A94E2F780FF10C023E333E34BEC51E499
:101A0000D7016D917D918D919C910E94C336F70114
:101A100060837183828393830F5F1F4FF4E0EF0E27
:101A2000F11C03301105F9F6D2CF8091F105813018
:101A300039F424E0521621F00E94941385E24AC63C
:101A40008CE0EEECF5E0DE011D9601900D928A959A
:101A5000E1F7A7FE17C08091F205873020F00E94C1
:101A600094138DE137C69091B505981759F0BE01D2
:101A7000635F7F4F0E949C21811104C00E949413D8
:101A800087E028C63091EB053F8F323021F03830A7
:101A900009F4A2C007C1511004C00E9494138AE146
:101AA00019C6C10180759927892B09F46FCF609100
:101AB0000B0670910C0680910D0690910E060E9407
:101AC00091370E94F934673050F6809106068431D0
:101AD00041F0823011F427FE04C00E94941384E187
:101AE000F9C5662319F061506F8F03C08091F2052C
:101AF0008F8FBE016F5F7F4F8F8D0E949C21882347
:101B000009F4BCCF409006066090E6057090E705AA
:101B10008090E8059090E905DE0111967D01F8E1DD
:101B2000AF2EF6E0BF2EA2ECCA2EA5E0DA2E00E022
:101B300010E0E52DF0E0FEA3EDA38DA19EA1002E07
:101B400002C0959587950A94E2F780FF33C0F4E1CF
:101B50004F1226C0D60158962D913D914D915C9122
:101B60005B976D917D918D919C910E94AB33F501B6
:101B700020813181428153810E94AB33D7016D9323
:101B80007D938D939C9313970230A1F4A40193014C
:101B90000E94AB33F70160837183828393830AC011
:101BA000F50180819181A281B381F70180839183C6
:101BB000A283B3830F5F1F4FF4E0EF0EF11C24E00C
:101BC000A20EB11C34E0C30ED11C0330110509F084
:101BD000B4CF9FEA29220AC1552009F45ECF609054
:101BE000E6057090E7058090E8059090E90508E12A
:101BF00016E0E2ECCE2EE5E0DE2E5E018DE0A80ED2
:101C0000B11CE12CF12CA52DB0E0B8A3AF8F8F8DC6
:101C100098A10E2C02C0959587950A94E2F780FF53
:101C200026C0F5012081318142815381D6016D9119
:101C30007D918D919C910E94AB33F801208131817F
:101C4000428153810E94AB33D8016D937D938D9374
:101C50009C931397B2E0EB1214C0A40193010E946D
:101C6000AB33F80160837183828393830AC0F601EA
:101C7000808D918DA28DB38DF80180839183A28395
:101C8000B383FFEFEF1AFF0A0C5F1F4F24E0C20E71
:101C9000D11C34E0A30EB11C83E0E816F10409F076
:101CA000B6CFA3C09E8D933079F4AF8DA53009F4E3
:101CB0008BC0A73009F491C0A33009F096C0BE01D3
:101CC0006F5F7F4F86E084C0552079F34090EF0529
:101CD0006090E6057090E7058090E8059090E90532
:101CE00072ECC72E75E0D72E08E116E05E01BDE06C
:101CF000AB0EB11CE12CF12CE52DF0E0FEA3EDA321
:101D00008DA19EA10E2C02C0959587950A94E2F7AD
:101D100080FD0BC0F60180819181A281B381F80121
:101D200080839183A283B3833EC0FF8DF730D9F1C6
:101D3000411028C0D60158962D913D914D915C914E
:101D40005B97F50160817181828193810E94AC3340
:101D5000D8012D913D914D915C910E94AC33F801D9
:101D60006083718382839383F2E0EF121CC0A4012D
:101D700093010E94AC33D8016D937D938D939C9316
:101D8000139711C0F6012081318142815381D8011E
:101D90006D917D918D919C910E94AC33F80160838F
:101DA000718382839383FFEFEF1AFF0A24E0C20E50
:101DB000D11C0C5F1F4F34E0A30EB11C83E0E8166A
:101DC000F10409F09DCF71CFBE016F5F7F4F87E0B7
:101DD0000E949C21811109C051CE8091EC05823076
:101DE00020F00E9494138EE175C41F8E1091EC05B3
:101DF000153059F4552009F4BFC1AE8DA13009F456
:101E000044C20E9494138FE165C4BE8DB23009F0C4
:101E1000B3C11123F1F020E030E0A9016091F60593
:101E20007091F7058091F8059091F9050E9485342D
:101E3000811104C00E94941386E14CC4143028F42C
:101E4000123058F4113029F020C2143009F453C173
:101E50001CC251101AC21E8E92C1552009F41DCE0B
:101E6000FFA1EF2FF0E0FEA3EDA338A5232F30E074
:101E70003BA72AA781E090E03C0108A402C0660CC1
:101E8000771C0A94E2F70FA002C0880F991F0A94EA
:101E9000E2F7682A792A852D90E086219721892BFF
:101EA00021F40E94941380E215C48DA19EA1880F95
:101EB000991F880F991FFC01E651FA4FDC01A155CB
:101EC000BA4F53962D913D914D915C91569766A5D1
:101ED00077A580A991A90E94AB336B017C018AA5EB
:101EE0009BA5880F991F880F991FFC01E651FA4F97
:101EF000DC01A155BA4F53962D913D914D915C91C6
:101F0000569766A577A580A991A90E94AB334B018E
:101F10005C0127FE40C0E89427F820911806309114
:101F2000190640911A0650911B066091C2057091E6
:101F3000C3058091C4059091C5050E948534811127
:101F400073C320911C0630911D0640911E065091CE
:101F50001F066091C6057091C7058091C8059091D4
:101F6000C9050E94853481115FC3209120063091FC
:101F7000210640912206509123066091CA05709176
:101F8000CB058091CC059091CD050E9485348823A6
:101F900009F49BC049C3F9A14F2E512C6420752030
:101FA000672821F40E94941383E294C321EF222234
:101FB0008091EE05813009F456C00AA51BA5000FDB
:101FC000111F000F111F06501A4FD8012D913D917E
:101FD0004D915C91C501B4010E94AB332B013C01D2
:101FE000ADA0BEA0AA0CBB1CAA0CBB1CF501E65000
:101FF000FA4F5F012081318142815381C701B601CF
:102000000E94AB33A30192010E949B286B017C01CB
:10201000D8012D913D914D915C91F50160817181C7
:10202000828193810E949B284B015C0160930F0683
:102030007093100680931106909312069B01AC01D9
:10204000C701B6010E94AB336B017C01E894F7F83D
:102050002AE037ED43EA5BE3C701B6010E94883608
:1020600018164CF112C18AEF682E85E0782E00E038
:1020700010E0C201002E02C0959587950A94E2F700
:1020800080FF10C023E333E34BEC51E4D3016D91A7
:102090007D918D919C910E94C336F3016083718381
:1020A000828393830F5F1F4FF4E06F0E711C033028
:1020B0001105F9F682CF20E030E040E05FE3C70190
:1020C000B6010E948836181624F40E94941381E207
:1020D00001C32FE632E143E85AE3C501B4010E948F
:1020E000C3369B01AC01C701B6010E9488361816A1
:1020F0000CF0CBC0EACF552009F4CFCC20911806C4
:102100003091190640911A0650911B066091C20544
:102110007091C3058091C4059091C5050E948534D6
:102120008111B3C020911C0630911D0640911E06FE
:1021300050911F066091C6057091C7058091C80532
:102140009091C9050E94853481119FC0209120067D
:102150003091210640912206509123066091CA05D4
:102160007091CB058091CC059091CD050E9485346E
:10217000882309F4AACF89C02E8D211186C0C10100
:102180008E7D9C7F85C0C301B2010E9450372B0118
:102190003C01A5019401C701B6010E949B289B0147
:1021A000AC01C301B20190580E948C342B013C0158
:1021B0008091EC05833021F477FA709477F870946D
:1021C00080910F0690911006A0911106B091120611
:1021D00089A39AA3ABA3BCA320E030E0A901BC0172
:1021E000CD010E94853487FF11C077FA709477F88B
:1021F000709489A19AA1ABA1BCA1B05880930F069D
:1022000090931006A0931106B09312060DA11EA183
:10221000000F111F000F111F06501A4FA30192014A
:10222000C501B4010E94C3369B01AC01C701B601D0
:102230000E94AB3320E030E040E05FE30E94C33611
:10224000D8016D937D938D939C9313970AA51BA53D
:10225000000F111F000F111F06501A4FA30192010A
:10226000C701B6010E94C3369B01AC01C501B40190
:102270000E94AC3320E030E040E05FE30E94C336D0
:10228000F8016083718382839383C1018E7D907E88
:10229000892B21F00E94941384E21CC28091ED05E9
:1022A0008093B0058091F6059091F705A091F8050F
:1022B000B091F9058093BD059093BE05A093BF052D
:1022C000B093C005C0901306D0901406E090150698
:1022D000F0901606A70196016091B9057091BA05B4
:1022E0008091BB059091BC050E9485348823D9F06C
:1022F000C092B905D092BA05E092BB05F092BC0538
:10230000809121079091220790FF04C08091EA05F7
:10231000811109C08091B805882329F020E0B70118
:10232000A6010E94DB13809117068093C10580915E
:10233000F5059091B8059817B9F08093B8052091EC
:1023400021073091220730FF04C09091EA059111D6
:102350000BC04091B9055091BA056091BB057091D1
:10236000BC0520E00E94DB138091F4059091B70535
:10237000981721F08093B7050E9437148091EB05E0
:10238000813051F460910B0670910C0680910D061E
:1023900090910E060E94DA078091F0058093B305B4
:1023A0008091EE058093B1053E8D3330F9F4809134
:1023B000F1058093B405813089F4809120069091D5
:1023C0002106A0912206B09123068093E605909302
:1023D000E705A093E805B093E90508C01092E6056B
:1023E0001092E7051092E8051092E9058091F20538
:1023F0009091B505981759F08093B5058CE0FE01D2
:102400003D96AEECB5E001900D928A95E1F7809192
:10241000EF058093B2058091EB0590E0FC013297C7
:10242000E830F10508F05FC0E75BFF4F0C94E93737
:10243000BE016F5F7F4F8F8D0E9480208091B50518
:102440009F8D891350C08CE0FE013196AEECB5E053
:102450002EC0AE8DAA2399F0E090B905F090BA0590
:102460000091BB051091BC05C090B80520E040E08C
:1024700050E060E87FEB88E196E00E948B04E090FA
:10248000B905F090BA050091BB051091BC05C0904C
:10249000B80520E040E050E060E87FEBCE01019617
:1024A0000E948B048CE0FE013196A2ECB5E0019015
:1024B0000D928A95E1F717C062EC75E086E003C0E3
:1024C00062EC75E087E00E9480200DC08CE0E8E1BE
:1024D000F6E0AAEDB5E0EBCF8CE0EAEDF5E0DF0148
:1024E0001D928A95E9F78091EC058093AF058530C0
:1024F00009F485C0BE8DB23009F081C08430E8F4A3
:10250000823008F040C0882351F1813009F06EC05C
:10251000E090B905F090BA050091BB051091BC059B
:102520004091BD055091BE056091BF057091C005F9
:10253000C090B8052091B00521C0843009F056C084
:102540004091BD055091BE056091BF057091C005D9
:102550002091B00588E196E00E94390847C0E090DC
:10256000B905F090BA050091BB051091BC05C0906B
:10257000B80520E040E050E060E87FEB88E196E0BD
:102580000E948B0433C0C090BD05D090BE05E09082
:10259000BF05F090C00500910F0610911006209124
:1025A0001106309112068091B8058F938091BC0579
:1025B0008F938091BB058F938091BA058F93809103
:1025C000B9058F93E9A5EF93F8A5FF938FA0A0908D
:1025D000B0054AEF55E068E176E082EC95E00E94B4
:1025E000ED040FB6F894DEBF0FBECDBF8CE0E8E17E
:1025F000F6E0A2ECB5E001900D928A95E1F78091AA
:10260000F3058093B605882369F00E944116109265
:10261000A1058091B605823019F40E94180902C004
:102620001092B60580E056C08091EE058130B1F47D
:1026300023E333E34BEC51E460910F0670911006F5
:1026400080911106909112060E94C33660930F0686
:1026500070931006809311069093120640900F0617
:1026600050901006609011067090120620E030E045
:1026700040E850E4C301B2010E94C336A3019201B5
:102680000E94C3362B013C01A7019601C701B60188
:102690000E94C3369B01AC01C301B2010E94AB335F
:1026A0002B013C01A5019401C501B4010E94C33670
:1026B0009B01AC01C301B2010E94AB332B013C0171
:1026C00020E030E0A9010E94853487FF5CCD0E94A4
:1026D000941382E2AB960FB6F894DEBF0FBECDBF67
:1026E000DF91CF911F910F91FF90EF90DF90CF90EE
:1026F000BF90AF909F908F907F906F905F904F9022
:102700003F902F900895E0EBF0E080818F778083F9
:102710002B9808958091B300882329F08091B00010
:1027200080688093B00008951092B300E0EBF0E071
:1027300080818F7780832B980895239A239A259AF6
:102740000C94941383E88093B000E1EBF0E0808177
:10275000887F8260808308958093B3000895CF922C
:10276000DF92EF92FF926B017C0120E030E04AE7BC
:1027700054E40E948836181634F4C12CD12C8AE710
:10278000E82E84E4F82E2CE53FE842E85EE3C7013A
:10279000B6010E94C33620E030E040E05FE30E94D3
:1027A000AC330E9462350E94F934862FFF90EF907F
:1027B000DF90CF9008951F93CF93DF9300D000D088
:1027C0001F92CDB7DEB7182F80919205823009F4A1
:1027D00040C0E0912107F0912207F0FF02C02111D3
:1027E0000CC029834A835B836C837D830E94C4155C
:1027F0007D816C815B814A812981E0912107F09183
:102800002207F0FF02C021110AC04A835B836C8358
:102810007D830E9441167D816C815B814A8111110B
:102820000AC00F900F900F900F900F90DF91CF91F3
:102830001F910C949413113011F42D9801C02D9A0E
:10284000CB01BA010E94AF138093B3000E94A21380
:102850002B9A0F900F900F900F900F90DF91CF91C8
:102860001F910895439808953B9A0C943214CF9386
:10287000DF931F92CDB7DEB790919205923079F039
:1028800089830E94C4150E9441168981823011F407
:10289000439A05C00F90DF91CF910C9432140F90A2
:1028A000DF91CF91089590910801809109018917D6
:1028B00008F48058891B0895E0ECF0E08081826084
:1028C00080831092C50080E18093C400E1ECF0E0C9
:1028D000808180618083808188608083808180683E
:1028E00080830895E091070191E09E0F903409F4F0
:1028F00090E020910601921305C02091930524FFDA
:10290000F8CF0895F0E0EC5DF94F808390930701D4
:102910008091C10080628093C10008951F920F9240
:102920000FB60F9211248F939F93EF93FF93809193
:102930000601E82FF0E0EC5DF94F90819093C6001E
:102940008F5F803409F480E0809306019091070145
:10295000891305C08091C1008F7D8093C100FF91D4
:10296000EF919F918F910F900FBE0F901F90189530
:102970009091080180910901891761F0E92FF0E039
:10298000EC59F94F80819F5F903809F490E0909363
:10299000080108958FEF08951F920F920FB60F92BE
:1029A00011242F933F934F935F936F937F938F9354
:1029B0009F93AF93BF93EF93FF938091C6008132B3
:1029C000B1F028F48831E1F40E9418092AC08F334D
:1029D00041F08E37A9F49FB7F894809193058260F7
:1029E0000BC09FB7F89480919305816005C09FB795
:1029F000F894809193058860809393059FBF11C0E0
:102A0000E091090191E09E0F903809F490E0209147
:102A10000801921731F0F0E0EC59F94F8083909360
:102A20000901FF91EF91BF91AF919F918F917F919C
:102A30006F915F914F913F912F910F900FBE0F902B
:102A40001F90189580910901809308010895CF93F4
:102A5000C0919305CC2309F48EC08C2F807649F168
:102A600081E0809392050E948313C6FF17C0C5FFC3
:102A700002C08FEF01C08DEF0E94422D81E00E94C5
:102A8000612D9FB7F894809193058F7E8093930575
:102A90009FBF8091930584FFFCCF03C08EEF0E94FF
:102AA000422D9FB7F894809193058F798093930579
:102AB0009FBFC4FF06C00E94831381E080939105ED
:102AC00061C0C0FF0AC00E94DC309FB7F8948091BB
:102AD00093058E7F809393059FBFC3FF15C08091A0
:102AE0009205803149F480E2809392050E946A1930
:102AF0000E948C191092A1059FB7F89480919305BC
:102B0000877F809393059FBFC1FF1FC0809192056F
:102B1000883099F480E1809392050E948A130E9484
:102B20008C190E945B168091210781FF04C081E00F
:102B30008093A10502C01092A1059FB7F8948091DF
:102B400093058D7F809393059FBFC2FF14C00E94A1
:102B50008924892B31F00E94831388E080939205A9
:102B600002C0109292059FB7F894809193058B7FD5
:102B7000809393059FBF80919205847319F0CF9144
:102B80000C948C19CF9108958091A105882341F070
:102B90009FB7F894809193058260809393059FBFBF
:102BA0000895CF93DF930E94872D80919205813005
:102BB00021F482E00E94612D21C0109292058AE0EA
:102BC00091E00E9441321AC08D3069F0DD2389F115
:102BD000D1E0893209F4D0E00E94B8148F3F09F4A3
:102BE00044C08A3089F7EC2FF0E0E65FFE4F108298
:102BF0000E94271580919105882311F0C0E0EBCF4A
:102C000080910A01811103C00E94F42CF7CF843215
:102C100029F48AE091E00E946032F6CF809192051B
:102C2000813011F489E0F0CF8AE091E00E94BD0983
:102C3000EBCF813288F28F3279F28832A1F0CF3433
:102C400028F08BE00E94F42CC0E0C6CF2C2F30E09F
:102C5000CF5F9FE9980FF901E65FFE4F9A3108F4C4
:102C600080528083B9CFD1E0B7CF0E94C4150E94B3
:102C7000271580919105882309F4AECFDF91CF917C
:102C800008950E94C41580919205803171F481E00D
:102C90008093A1050AC080919205803159F40E9469
:102CA000271580919105811105C00E948924892BE7
:102CB000B1F7F1CF08958091210782FF02C0289AD1
:102CC00001C02898809192058471A1F080918A01B9
:102CD00080939E0180918B0180939D0180911407C8
:102CE000880F8450819580939C0180916F00826051
:102CF00080936F00089580916F008D7F80936F00A7
:102D000080918100887F8160809381001092890189
:102D1000809117078F3F21F49091930595FF09C08B
:102D200090919205943029F090E00E94902881E0E3
:102D300001C080E09091210792FF02C091E08927B5
:102D4000882311F0289A0895289808951F920F92C9
:102D50000FB60F9211242F933F934F935F936F936E
:102D60007F938F939F93AF93BF93EF93FF93809144
:102D700089018111FEC19BB180919E01807E9F716E
:102D8000892B8BB98BB1837E90919D01892B8BB957
:102D900080919C0186BD82E085BD81E080938901A0
:102DA00078948091B0019091B101892B09F0B3C062
:102DB00080918E0190918D01981709F4A1C0E09146
:102DC0008E0186E0E89FF0011124EE54FE4FF0934F
:102DD000B101E093B0018381948190938900809345
:102DE0008800808191819093AC018093AB01E28156
:102DF0008091AD018E17C1F1E093AD0183E1E89FB1
:102E0000F0011124EA52FE4FF093AF01E093AE01BE
:102E100085859685A785B089B695A7959795879559
:102E200080938F0190939001A0939101B0939201B0
:102E30008093930190939401A0939501B093960190
:102E40008093970190939801A0939901B0939A0170
:102E5000809121079091220790FF06C082898823E4
:102E600019F081890E94AC13E091AE01F091AF019D
:102E700080918A019081892780939E01A091B00161
:102E8000B091B10115962C9181819281A381B48179
:102E9000022E04C0B695A795979587950A94D2F708
:102EA00080939F019093A001A093A101B093A201F0
:102EB00085819681A781B085022E04C0B695A7951D
:102EC000979587950A94D2F78093A3019093A401D4
:102ED000A093A501B093A60181859285A385B485B1
:102EE00004C0B695A795979587952A95D2F78093B4
:102EF000A7019093A801A093A901B093AA010BC0C8
:102F00000E947B169FB7F89480919305846080930C
:102F100093059FBF2EC10E94DB2C10929D018091D2
:102F20009F019091A001A091A101B091A2014091B7
:102F30008F01509190016091910170919201840FE5
:102F4000951FA61FB71F80938F0190939001A093A8
:102F50009101B0939201E091AE01F091AF014585EE
:102F6000568567857089481759076A077B0768F592
:102F700024E020939D014585568567857089841BD3
:102F8000950BA60BB70B80938F0190939001A093A4
:102F90009101B093920120818091950590919605C1
:102FA000A0919705B091980525FF04C00197A1094C
:102FB000B10903C00196A11DB11D809395059093A1
:102FC0009605A0939705B09398058091A3019091E1
:102FD000A401A091A501B091A60140919301509147
:102FE00094016091950170919601840F951FA61F21
:102FF000B71F8093930190939401A0939501B09390
:1030000096014585568567857089481759076A076F
:103010007B0778F520919D01286020939D014585CF
:10302000568567857089841B950BA60BB70B80931B
:10303000930190939401A0939501B0939601208100
:103040008091990590919A05A0919B05B0919C055E
:1030500026FF04C00197A109B10903C00196A11D73
:10306000B11D8093990590939A05A0939B05B09309
:103070009C058091A7019091A801A091A901B09110
:10308000AA01409197015091980160919901709126
:103090009A01840F951FA61FB71F809397019093E5
:1030A0009801A0939901B0939A014585568567854B
:1030B0007089481759076A077B0778F520919D01A9
:1030C000206120939D014585568567857089841B05
:1030D000950BA60BB70B8093970190939801A09343
:1030E0009901B0939A01208180919D0590919E0550
:1030F000A0919F05B091A00527FF04C00197A109E9
:10310000B10903C00196A11DB11D80939D05909347
:103110009E05A0939F05B093A005809192058430F1
:1031200039F48091940590919D01892380939D01AC
:103130008091AB019091AC0101979093AC01809389
:10314000AB01892B69F41092B1011092B00180910A
:103150008E018F5F80938E01863011F410928E0164
:1031600080918B0190919D01892780939D01109200
:103170008901FF91EF91BF91AF919F918F917F91C5
:103180006F915F914F913F912F910F900FBE0F90D4
:103190001F9018951F920F920FB60F9211248F93C4
:1031A0009F939BB180918B018C71937E892B8BB9FE
:1031B00015BC9F918F910F900FBE0F901F90189587
:1031C000FF920F931F93CF93DF9310928B01109276
:1031D0008A01C0E0D0E00C2F1C2F2091150730E0B1
:1031E0008C2F0C2E02C0359527950A94E2F720FF0C
:1031F00007C0F0908B010E942B238F2980938B01B5
:103200002091160730E002C0359527951A95E2F710
:1032100020FF08C010918A01802F0E943523812B46
:1032200080938A012196C330D105A9F6DF91CF9111
:103230001F910F91FF9008950E947B168BE2EAE5A3
:10324000F1E0DF011D928A95E9F783E2EFE8F1E012
:10325000DF011D928A95E9F710928801109287018B
:1032600010928E0110928D0181E080938C0110925A
:1032700089010E94E0188BB1837E90918B01892B8C
:103280008BB98BB18F7190918A01892B8BB908957D
:103290008AB18C618AB9209A8AB1806E8AB9E1E8D4
:1032A000F0E080818F7E8083808188608083E0E889
:1032B000F0E080818C7F808380818F708083EEE658
:1032C000F0E08081887F808314BC15BC80818160A0
:1032D00080830895CF93DF93C0918701D0918801B7
:1032E0002097B9F081E080935B016091710170914A
:1032F000720180917301909174019B01AC010E9455
:10330000C3366E8B7F8B888F998F109288011092B5
:103310008701DF91CF9108952F923F924F925F9254
:103320006F927F928F929F92AF92BF92CF92DF92D5
:10333000EF92FF920F931F93CF93DF93CDB7DEB73A
:10334000E5970FB6F894DEBF0FBECDBF90918E010A
:1033500080918C01981709F4FDC5809187019091A7
:103360008801892B09F073C20E948924FC01909383
:10337000880180938701009709F4ECC580915B0177
:10338000882319F010925B01D3C080915A018F5F9E
:10339000853019F080935A0102C010925A010091B1
:1033A0005A0123E1209F800111240A521E4F1093DD
:1033B0008601009385018581D8018C9346815781D0
:1033C0006085718593E0440F551F661F771F9A959E
:1033D000D1F711964D935D936D937C93149742852D
:1033E00053856485758523E0440F551F661F771F3D
:1033F0002A95D1F715964D935D936D937C9318970D
:10340000468557856089718933E0440F551F661FD3
:10341000771F3A95D1F719964D935D936D937C93F1
:103420001C97428953896489758983E0440F551F2D
:10343000661F771F8A95D1F71D964D935D936D9307
:103440007C935097848152968C93608171818281A4
:1034500093810E94AF13F801818B00918701109135
:103460008801D80152966D917D918D919C915597CF
:103470000E94253560935C0170935D0180935E012D
:1034800090935F01F80122A533A544A555A50E949C
:103490008C349B01AC016093600170936101809357
:1034A00062019093630160E070E080EA9FE30E9414
:1034B0008C346093640170936501809366019093EE
:1034C0006701109268011092690110926A011092CE
:1034D0006B01809192058032E1F4609179017091E5
:1034E0007A0180917B0190917C01609371017093CE
:1034F000720180937301909374019B01AC010E944F
:10350000C336D80156966D937D938D939C935997AE
:103510000FC0F80166897789808D918D0E945037A0
:1035200060937101709372018093730190937401A1
:1035300010926D0110926E0110926F011092700145
:103540000091870110918801D80196968D909D90E9
:10355000AD90BC909997A501940160E070E080E087
:103560009FE30E948C342B013C0180919205F8016D
:10357000C2A4D3A4E4A4F5A4803209F04FC0F2E0C1
:10358000F0936C01D80156962D913D914D915C912F
:1035900059972D833E834F835887C301B2010E9400
:1035A000C3369B01AC01C701B6010E94AB332B01AE
:1035B0003C0120E030E0A9010E94853487FF1DC056
:1035C000A5019401C501B4010E94AC33A701960185
:1035D0000E94C3369B01AC016D817E818F819885ED
:1035E0000E94AB330E9450376093790170937A0147
:1035F00080937B0190937C012AC140926D0150928F
:103600006E0160926F0170927001109279011092B8
:103610007A0110927B0110927C0119C110926C0109
:10362000C0927D01D0927E01E0927F01F0928001F4
:103630000E9499244B015C016093790170937A0197
:1036400080937B0190937C019B01AC010E94C33667
:1036500069837A838B839C83009187011091880111
:10366000D8019A962D913D914D915C919D97298716
:103670003A874B875C8756962D913D914D915C9191
:1036800059972D833E834F8358879B01AC016D81F1
:103690007E818F8198850E94AB339B01AC01C30171
:1036A000B2010E94C3369B01AC0169857A858B8586
:1036B0009C850E94AC3320E030E040E05FE30E9454
:1036C000C3366B017C0120E030E0A9010E948836FE
:1036D00018160CF0ACC029853A854B855C85C7016E
:1036E000B6010E94853487FF8EC0F80182A093A0A6
:1036F000A4A0B5A029813A814B815C81C501B401A8
:103700000E94AB339B01AC01C301B2010E94C336DE
:10371000609381017093820180938301909384016F
:10372000A70196010E94853487FF3DC0C501B40101
:103730000E945037609375017093760180937701F2
:1037400090937801A50194016D817E818F81988588
:103750000E948534811104C0F1E0F0936C0177C0C0
:103760002D813E814F815885C501B4010E94AB3344
:103770009B01AC01C301B2010E94C3369B01AC01A5
:1037800060917D0170917E0180917F019091800117
:103790000E94AB3360937D0170937E0180937F0123
:1037A0009093800154C0C0927D01D0927E01E0923E
:1037B0007F01F0928001C0928101D0928201E0925B
:1037C0008301F0928401D80196966D917D918D913F
:1037D0009C9199979B01AC010E94AC33A701960183
:1037E0000E94C33629813A814B815C810E94AC33AF
:1037F0000E94503760937501709376018093770132
:103800009093780124C0B2E0B0936C018091710173
:1038100090917201A0917301B09174018093750130
:1038200090937601A0937701B093780110C0109225
:103830007D0110927E0110927F0110928001809292
:10384000750190927601A0927701B09278018091F3
:103850008D01F6E0F89FF0011124EE54FE4FFE8337
:10386000ED8380915A0182832091870130918801F4
:103870003E872D87D9019A96BC91BCA7F901F3A583
:10388000FDA7D9019C96BC91BEA7F901F5A5FFA79C
:10389000209164013091650140916601509167016A
:1038A0006CA57DA58B2F9F2F0E94AB3368A779A7AE
:1038B0008AA79BA720E030E0A9010E94853487FFFA
:1038C00004C018A619A61AA61BA620917D01288F50
:1038D00030917E01398F40917F014A8F5091800154
:1038E0005B8F809175018C8F909176019D8FA09157
:1038F0007701AE8FB0917801BF8FE0918101E8A38D
:10390000F0918201F9A3209183012AA330918401CF
:103910003BA340916D014CA350916E015DA380913A
:103920006F018EA3909170019FA320917901309136
:103930007A0140917B0150917C0128AB39AB4AABB5
:103940005BAB3091710139834091720149872090BE
:1039500073013090740150916C015F878CA58C8B42
:103960009DA59D8BAEA5AE8BBFA5BF8B8EE3C82E4C
:1039700083ECD82E8EE2E82E89E3F82E188A198A75
:103980001A8A1B8A26013701EF85EE2321F0E130E8
:1039900009F47CC0B1C0AD85BE8596962D913D9150
:1039A0004D915C919997C701B6010E94C3364B01B6
:1039B0005C0120E030E040E05FE30E94C3369B0101
:1039C000AC0169817985C1010E94AC339B01AC01D6
:1039D000C701B6010E94C3369B01AC016C897D8989
:1039E0008E899F890E94AB338B018DAB9CAB288D58
:1039F000398D4A8D5B8D0E94853487FF3FC0288DAD
:103A0000398D4A8D5B8D6CA57DA58EA59FA50E94E5
:103A1000AB339B01AC010E94AC336B017C012C8D5C
:103A20003D8D4E8D5F8D69817985C1010E94AC33DA
:103A30009B01AC01C701B6010E948C346B017C0173
:103A400028A139A14AA15BA1688D798D8A8D9B8DB2
:103A50000E948534882319F0B1E0BF8702C0E2E0FC
:103A6000EF87FC8DF9832D8D29872E8C3F8C088D57
:103A7000198D3A8D3DAB4B8D4CABAFC0A501940178
:103A800069817985C1010E94AC337CC0A701960190
:103A90006C8D7D8D8E8D9F8D0E94C3369B01AC01F8
:103AA0006C897D898E899F890E94AB338B018DAB98
:103AB0009CAB28A139A14AA15BA10E94853487FF54
:103AC0008CC028A139A14AA15BA16C897D898E890E
:103AD0009F890E94AB332C8D3D8D4E8D5F8D0E9452
:103AE0008C346B017C0108A119A15AA15DAB8BA19B
:103AF0008CAB92E09F8771C0AD85BE8596962D9167
:103B00003D914D915C919997C701B6010E94C336D2
:103B10004B015C019B01AC0169817985C1010E9467
:103B2000883618169CF520E030E040E05FE3C501E0
:103B3000B4010E94C3369B01AC0169817985C10142
:103B40000E94AB339B01AC01C701B6010E94C33692
:103B50009B01AC016C897D898E899F890E94AB3362
:103B60008B018DAB9CAB2CA13DA14EA15FA10E940E
:103B7000883618165CF4A501940169817985C10124
:103B80000E94AB33698379871C0127C02CA13DA11A
:103B90004EA15FA16C897D898E899F890E94AB337C
:103BA0009B01AC010E94AC336B017C0128A939A9AF
:103BB0004AA95BA969817985C1010E94AC339B0147
:103BC000AC01C701B6010E948C346B017C010CA1D1
:103BD0001DA1BEA1BDABEFA1ECABA7019601688909
:103BE00079898A899B890E94AC33688B798B8A8B0F
:103BF0009B8BA30192010E94853487FD5AC028A5A2
:103C000039A54AA55BA5B8018DA99CA90E94883653
:103C100018160CF444C089819985D10180937101F3
:103C200090937201A0937301B0937401FF85F09398
:103C30006C01409060015090610160906201709051
:103C4000630198014DA95CA9C301B2010E94C3366A
:103C500069837A838B839C830E9472346B017C011D
:103C600060915C0170915D0180915E0190915F01B6
:103C70000E9472344B015C01A70196010E94AB3394
:103C80000E94F93469877A878B879C87E985FA8552
:103C9000AD81BE81ED93FC933097B1F15AC02EE314
:103CA00033EC4EE259E3C301B2010E94AC332B0165
:103CB0003C01288939894A895B89C301B2010E9484
:103CC000AB336B017C012CA13DA14EA15FA1B801DA
:103CD0008DA99CA90E94883618167CF08981998547
:103CE000D1018093710190937201A0937301B093FD
:103CF00074013F8530936C019CCF0C8B1D8B4DA9BB
:103D00004E8B5CA95F8B40CE80919205803209F585
:103D1000109271011092720110927301109274014D
:103D2000109268011092690110926A0110926B0161
:103D3000C0925C01D0925D01E0925E01F0925F0161
:103D4000A3019201C701B6010E948C34AD85BE85E6
:103D5000EEC0209168013091690140916A01509153
:103D60006B01688979898A899B890E94AC332B0110
:103D70003C0129813A814B815C81C501B4010E94DB
:103D8000AB339B01AC01C301B2010E948C344B01E7
:103D90005C0129813A814B815C81C701B6010E9497
:103DA000AB33A50194010E94C33660936801709300
:103DB000690180936A0190936B0120EC31EE44E637
:103DC0005EE4C501B4010E94C3360E9472340E94B1
:103DD000F934603DB7E07B078105910520F4ED8162
:103DE000FE81158231C0603AFFE07F0781059105B1
:103DF00010F4E1E009C06034FFE17F07810591051F
:103E000010F4E2E001C0E3E0AD81BE811596EC93D1
:103E1000AD81BE8115962C911597022E04C0969502
:103E20008795779567950A94D2F7E985FA8502C058
:103E3000EE0FFF1F2A95E2F7ED93FC9361157105D4
:103E4000F1E08F07910538F4AD81BE8114967C9323
:103E50006E93139706C02FEF3FEFED81FE81348301
:103E6000238380918C0180938D018F5F863019F0C0
:103E700080938C0102C010928C0120916D013091D1
:103E80006E0140916F0150917001B8018DA99CA9FC
:103E90000E9488361816C4F4E0918701F0918801D9
:103EA000C801ADA9BCA982A793A7A4A7B5A789817A
:103EB0009A81AB81BC8180935C0190935D01A0935A
:103EC0005E01B0935F0142CA20E030E0A901B80171
:103ED0008DA99CA90E9488361816ACF51092710124
:103EE0001092720110927301109274011092680185
:103EF0001092690110926A0110926B01C0925C01EC
:103F0000D0925D01E0925E01F0925F010091870125
:103F1000109188012091600130916101409162010E
:103F200050916301C701B6010E948C34D8019A9662
:103F30006D937D938D939C939D970E94D62788E0E7
:103F40008093920507C010928801109287010E9409
:103F50007524FCC9E5960FB6F894DEBF0FBECDBF41
:103F6000DF91CF911F910F91FF90EF90DF90CF9055
:103F7000BF90AF909F908F907F906F905F904F9089
:103F80003F902F900895F999FECF92BD81BD81E0B9
:103F90008FBB80B50895F894F999FECF92BD81BD8D
:103FA00081E08FBB40B54627842F992787FD9095E8
:103FB000262F30E082239323892B39F06F3F19F0AD
:103FC00060BD84E006C084E104C0442321F060BDEC
:103FD00084E28FBBF99A789408959F92AF92BF9232
:103FE000CF92DF92EF92FF920F931F93CF93DF93C5
:103FF0008C017A016B01C40ED51EEB01912C5C0182
:10400000A61AB70ACE018A0D9B1DCC15DD0591F0CD
:10401000911009C0692D772767FD7095272F221F02
:104020002227221F01C021E06991922E960E0E9444
:10403000CB1FE8CF692DC8018E0D9F1DDF91CF9159
:104040001F910F91FF90EF90DF90CF90BF90AF90B6
:104050009F900C94CB1F9F92AF92BF92CF92DF9212
:10406000EF92FF920F931F93CF93DF938B017A010F
:104070006C01C40ED51EEC01912C5B01A81AB90A83
:10408000C5018C0F9D1FCC15DD0591F00E94C31F4B
:10409000911009C0292D332727FD3095232F221F8A
:1040A0002227221F01C021E0922E980E8993E8CF8B
:1040B000C8018E0D9F1D0E94C31F21E030E098169D
:1040C00011F020E030E0C901DF91CF911F910F91F5
:1040D000FF90EF90DF90CF90BF90AF909F900895AA
:1040E00021E5829FC001112440E550E09D5F0C94C2
:1040F000ED1F40E550E0BC018EEA93E00C94ED1F0B
:104100002DE0829FC00111244CE050E09E5F0C9492
:10411000ED1F69E080E090E00E94CB1F4EE450E08C
:1041200064EE76E081E090E00C94ED1F8AE08093ED
:10413000140789E1809317071092150781E0809397
:10414000160723E0209318078AE097EDA3EABCE363
:104150008093190790931A07A0931B07B0931C072D
:104160008FE692E1A3E0BBE380931D0790931E07C7
:10417000A0931F07B09320072093230780E090E0CF
:10418000A8ECB1E48093240790932507A093260719
:10419000B093270780E090E0AAEFB4E4809328076B
:1041A00090932907A0932A07B0932B0784E690E009
:1041B00090932D0780932C0780E090E0A0E8BFE368
:1041C00080932E0790932F07A0933007B093310769
:1041D00082E391E0909322078093210780E090E0B2
:1041E000A8ECB2E48093E4069093E506A093E6067B
:1041F000B093E7068093E8069093E906A093EA0659
:10420000B093EB068093EC069093ED06A093EE0638
:10421000B093EF0680E090E4ACE9B5E48093F0065B
:104220009093F106A093F206B093F3068093F40600
:104230009093F506A093F606B093F7068093F806E0
:104240009093F906A093FA06B093FB0680E09FECEA
:10425000A9E1BAE48093FC069093FD06A093FE06C4
:10426000B093FF068093000790930107A093020785
:10427000B093030780E098ECAFEAB8E480930407BA
:1042800090930507A0930607B093070780E090E09E
:10429000ABE5B3EC8093080790930907A0930A0756
:1042A000B0930B0780E090E0A6E9B3EC80930C0795
:1042B00090930D07A0930E07B0930F0780E090E056
:1042C000A0E2B1EC8093100790931107A09312071E
:1042D000B09313070C9489201F93CF93DF93182F6B
:1042E000EB0181E5189FB00111247D5F40E550E0AE
:1042F000CE010E942B20892B39F41882BE01812F18
:104300000E94702080E001C081E0DF91CF911F9179
:104310000895CF93DF93EC0140E550E06EEA73E03F
:104320000E942B20892B21F41882CE010E94792033
:1043300081E0DF91CF9108951F93CF93DF93182FE2
:10434000EB018DE0189FB00111247E5F4CE050E03E
:10435000CE010E942B20892B59F48CE0FE01119292
:104360008A95E9F7BE01812F0E94802080E001C07C
:1043700081E0DF91CF911F91089580E090E00E944D
:10438000C31F893059F44EE450E061E070E084EEE0
:1043900096E00E942B2021E0892B09F420E0822F57
:1043A0000895CF92DF92EF92FF92CF93DF93C82FC1
:1043B0006A017B0120E030E0A901C701B6010E943B
:1043C000853487FD0BC1C43608F445C02CE92C0F99
:1043D00080E02330B8F530E0823079F0F901EE0F5B
:1043E000FF1FEE0FFF1F833011F1813019F0EC51E8
:1043F000F94F23C0E051F94F20C0E901CC0FDD1F78
:10440000CC0FDD1FC450D94F20E030E040E752E42C
:10441000C701B6010E94C33620E030E040E752E415
:104420000E94C336688379838A839B83D3C0E85F05
:10443000F84FF7FAF094F7F8F094C082D182E28254
:10444000F382C8C08F5F2A3008F4CAC0843009F4F0
:10445000C7C02A50BECFC701B6010E9491370E9443
:10446000F9348C2F90E08932910508F0B9C0FC0135
:10447000EF5AFF4F0C94E937633008F4B3C06093F0
:104480001407A8C060931707A5C06093150702C062
:10449000609316070E94E0189DC0809121079091BB
:1044A0002207662311F0846091C08B7F8FC08091BA
:1044B000210790912207662311F0806487C08F7BCB
:1044C00085C08091210790912207662311F08068B2
:1044D0007DC08F777BC060931807C0921907D09278
:1044E0001A07E0921B07F0921C0774C0C0921D07C8
:1044F000D0921E07E0921F07F09220076BC08091B8
:10450000210790912207662311F081605FC08E7FA2
:104510005DC08091210790912207662311F082608F
:1045200055C08D7F53C0809121079091220766234B
:1045300021F084FF59C0806249C08F7D47C08091BF
:10454000210790912207662311F0886001C0877FC0
:1045500090932207809321070E94CC283BC0809132
:10456000210790912207662311F080612FC08F7C74
:104570002DC0609323072EC0C0922407D092250738
:10458000E0922607F092270725C0C0922807D09214
:104590002907E0922A07F0922B071CC070E0709365
:1045A0002D0760932C0716C0C0922E07D0922F07BC
:1045B000E0923007F09231070DC080912107909171
:1045C0002207662311F0916001C09E7F909322071D
:1045D000809321070E94892080E007C084E005C005
:1045E00083E003C086E001C08AE0DF91CF91FF90B5
:1045F000EF90DF90CF9008951F93CF93DF93CDB7C7
:10460000DEB72C970FB6F894DEBF0FBECDBF0E9469
:10461000BD21811107C087E00E94F42C0E949620E2
:104620000E948F2D10E0BE016F5F7F4F812F0E948F
:104630009C21811103C087E00E94F42C1F5F183079
:1046400091F72C960FB6F894DEBF0FBECDBFDF9169
:10465000CF911F910895882321F0813021F488E0C3
:10466000089584E0089580E10895882321F0813041
:1046700021F480E4089580E2089580E80895882375
:1046800021F0813021F484E0089582E0089580E1F2
:1046900008954F925F926F927F928F929F92AF9206
:1046A000BF92CF92DF92EF92FF920F931F93CF931F
:1046B000DF9310915302111101C012E111500091CA
:1046C0005102101709F4EFC08EE2189FE001112487
:1046D000CB5ADD4F8A8C9B8CAC8CBD8C6EA17FA19C
:1046E00088A599A59B01AC010E94AC332AA53BA5E6
:1046F0004CA55DA50E94C3366B017C019B01AC01FA
:10470000B401C5010E94853487FF02C064017501B0
:10471000A601B7014E8B5F8B688F798F111101C095
:1047200012E177247A94710E701619F02EE2622E3F
:1047300027C080915402081351C00E946A194EC0CC
:10474000679C800111240B5A1D4F711002C092E129
:10475000792E7A9480915402781202C00E946A19CC
:10476000F801C28CD38CE48CF58CA7019601668984
:104770007789808D918D0E948534811106C0E80172
:10478000809151027812DCCF29C0F80166A177A18F
:1047900080A591A59B01AC010E94AC33F80122A534
:1047A00033A544A555A50E94C3362E893F89488D5F
:1047B000598D0E94AC334B015C01A70196010E9408
:1047C0008534F80187FF05C0868A978AA08EB18E4E
:1047D000D6CFC68AD78AE08EF18ED1CF60905102B3
:1047E000FEE26F9E800111240B5A1D4F77247394B3
:1047F000760C82E1781201C0712C509053028EE247
:10480000482E751409F44DC0479CE0011124CB5A81
:10481000DD4FF80186889788A08CB18CCE88DF8820
:10482000E88CF98CA7019601C501B4010E9485347A
:1048300087FF23C0F80166A177A180A591A59B0100
:10484000AC010E94AC33F80122A533A544A555A5BF
:104850000E94C3369B01AC01C501B4010E94AC3378
:104860004B015C01A70196010E94853487FF05C0BA
:104870008E8A9F8AA88EB98E672C2A8D3B8D4C8D8F
:104880005D8D6E897F89888D998D0E948534811117
:1048900001C0672C7394F2E17F1201C0712C8E016C
:1048A000B0CF60925102DF91CF911F910F91FF9095
:1048B000EF90DF90CF90BF90AF909F908F907F90C0
:1048C0006F905F904F9008958CE1E5E3F2E0DF0197
:1048D0001D928A95E9F7109254021092530281E0DA
:1048E0008093520210925102089590915402809147
:1048F0005302891769F081E0890F823109F480E061
:1049000020915102921302C080935102809354026D
:1049100008958091540290915302981739F02EE235
:10492000829FC00111248B5A9D4F089580E090E032
:104930000895E0915402EF5FE23109F4E0E08091E4
:104940005302E81761F08EE2E89FF0011124EB5A60
:10495000FD4F66897789808D918D0C94503760E08A
:1049600070E0CB01089581E02091540290915202B1
:10497000291380E008952F923F924F925F926F9299
:104980007F928F929F92AF92BF92CF92DF92EF92DF
:10499000FF920F931F93CF93DF93CDB7DEB7AD9701
:1049A0000FB6F894DEBF0FBECDBF4B8F5C8F6D8FFF
:1049B0007E8FB22E209153023EE2239F10011124DC
:1049C000F101EB5AFD4F1F01E082F1820283138354
:1049D000C482128A138A148A158A12A613A614A6F0
:1049E00015A6158249E956E766E97EE746A357A36F
:1049F00060A771A76C0104EE16E09E01235F3F4F94
:104A000038A32F8F85E392E09AA389A37F01FE014B
:104A100031964F01A12CF601619171918191919193
:104A20006F01F80120813181428153810E94C33698
:104A30000E949336EF8DF8A16193719381939193C6
:104A4000F8A3EF8FE9A1FAA1419051906190719084
:104A5000FAA3E9A364197509860997092B013C019A
:104A600097FF07C0442455243201461A570A680AA2
:104A7000790AF7014682578260867186F1012289A0
:104A8000338944895589421653066406750610F425
:104A900029013A01F101428A538A648A758A0E9487
:104AA0002735F80120813181428153810E948C3465
:104AB0002B013C01F40161937193819391934F0118
:104AC00020E030E0A9010E94853487FF0AC0F1018F
:104AD00095818A2D9DA70E9435239DA5892BF101E3
:104AE0008583A3019201C301B2010E94C336F10183
:104AF00022A533A544A555A50E94AC33F10162A7B8
:104B000073A784A795A7A3940C5F1F4FF4E0EF0E43
:104B1000F11C23E0A2127FCF0E9450376B017C0171
:104B2000F10162A773A784A795A782899389A489B5
:104B3000B589892B8A2B8B2B09F4E5C120E030E065
:104B4000A9016B8D7C8D8D8D9E8D0E94853487FD96
:104B500021C0BB2061F02B8D3C8D4D8D5E8DC7013A
:104B6000B6010E948C346B8F7C8F8D8F9E8F20E0DE
:104B700030E040E85FE36B8D7C8D8D8D9E8D0E94D3
:104B8000853487FF0FC01B8E1C8E90E89D8FEFE34E
:104B9000EE8F08C0F9E9FB8F26E72C8F36E93D8FB1
:104BA0008EE78E8FA701960160E070E080E89FE3BA
:104BB0000E948C3469A77AA78BA79CA721E432E0D6
:104BC0003CA32BA380EF96E09AA389A3FE013D9618
:104BD000FA8FE98F9E012F5F3F4F38A32F8FC12C93
:104BE000D12C7601EF8DF8A180809180A280B380D6
:104BF00020E030E0A901C501B4010E94853488237A
:104C000009F483C029A53AA54BA55CA5C501B4014B
:104C10000E94C3364B015C01EF8DF8A16083718364
:104C2000828393839B01AC0160E070E080E89FE3A6
:104C30000E948C342B013C01E89477F8E9A1FAA199
:104C40002081318142815381C301B2010E94C33668
:104C50006DA37EA38FA398A79B01AC016B8D7C8D68
:104C60008D8D9E8D0E94853487FF08C0FB8DFDA32E
:104C70002C8D2EA33D8D3FA38E8D88A7F101F6A12B
:104C8000FB8FF101F7A1FC8FF101F0A5FD8FF10180
:104C9000F1A5FE8FE9A1FAA12485358546855785C2
:104CA000C301B2010E94C3363B018C019B01AC01E0
:104CB0006B8D7C8D8D8D9E8D0E94853487FF04C009
:104CC0006B8C7C8C0D8D1E8DC301D801F10186A3E8
:104CD00097A3A0A7B1A7EBA1FCA1208131814281BC
:104CE0005381C501B4010E94C3369B01AC01C701C9
:104CF000B6010E94AB336B017C01FDA1FB8F2EA19D
:104D00002C8F3FA13D8F88A58E8FEF8DF8A1349613
:104D1000F8A3EF8F2BA13CA12C5F3F4F3CA32BA30B
:104D200089A19AA104969AA389A3298D3A8DE217A5
:104D3000F30709F057CF90915302809154029813D2
:104D40000AC0F101168A178A108E118E168E178EE0
:104D500010A211A249C0A701960160E070E080E8AE
:104D60009FE30E94AB3320E030E040E05FE30E942D
:104D7000C3360E9450376B017C0120911907309196
:104D80001A0740911B0750911C07F10166A177A1FA
:104D900080A591A50E94C336A70196010E94C33643
:104DA0004B015C01A701960160E070E080E89FE3A1
:104DB0000E94AB339B01AC01C501B4010E948C344D
:104DC0007B018C0120E030E0A9010E94853487FF3F
:104DD00004C0E12CF12C00E010E0A701B801F101C2
:104DE000468F578F60A371A32B8D3C8D4D8D5E8DAB
:104DF0006B8D7C8D8D8D9E8D0E94C336162F072F57
:104E0000F82EE92E862F902FAF2DBE2DF10182A313
:104E100093A3A4A3B5A3A68CB78CC0A0D1A0609087
:104E20004D0270904E0280904F029090500293017C
:104E3000A401612F702F8F2D9E2D0E94853487FD38
:104E40000BC09301A401B501C6010E94853487FD02
:104E500011C0530164010EC0212F302F4F2D5E2D44
:104E6000B501C6010E94853487FD04C0A12EB02E75
:104E7000CF2CDE2CC501D601F101828F938FA48F38
:104E8000B58F8CE0FE013196A1E4B2E001900D9265
:104E90008A95E1F7812F902FAF2DBE2D80934D0283
:104EA00090934E02A0934F02B09350028CE0FE010B
:104EB0003D96A5E3B2E001900D928A95E1F78091CD
:104EC0005202809353028F5F823109F480E0809315
:104ED0005202AD960FB6F894DEBF0FBECDBFDF9184
:104EE000CF911F910F91FF90EF90DF90CF90BF90E7
:104EF000AF909F908F907F906F905F904F903F907A
:104F00002F900C944923AD960FB6F894DEBF0FBED8
:104F1000CDBFDF91CF911F910F91FF90EF90DF9068
:104F2000CF90BF90AF909F908F907F906F905F9049
:104F30004F903F902F900895809195059091960500
:104F4000A0919705B0919805809335029093360211
:104F5000A0933702B09338028091990590919A05F9
:104F6000A0919B05B0919C058093390290933A02E1
:104F7000A0933B02B0933C0280919D0590919E05C9
:104F8000A0919F05B091A00580933D0290933E02B1
:104F9000A0933F02B09340020895809153029091F4
:104FA0005402891708F48E5E891B08950E946A19BD
:104FB00080915402809351020C9449236F927F9206
:104FC0008F929F92AF92BF92CF92DF92EF92FF9219
:104FD0000F931F93CF93DF937C018B016A01FB0139
:104FE0008081F701E80FF11D2081EF012D3229F4B6
:104FF000229621816624639407C02B3211F02196FA
:1050000002C022962181612CA12CB12C712C60E070
:1050100070E0CB01FE0130ED932E920E29E02915B0
:10502000C8F0B39428E02B1588F0A1107A94A5E07D
:10503000B0E09B01AC010E94B037660F771F881F5C
:10504000991F690D711D811D911D0BC0A11009C013
:10505000739407C02EEF921207C0A11005C0AA24B6
:10506000A39421962081D6CFBB2009F449C00E9489
:1050700025354B015C0120E030E0A9010E94853418
:10508000882361F18FEF78166CF42AE037ED43E264
:105090005CE3C501B4010E94C3364B015C0173940B
:1050A0007394F0CF78120BC02DEC3CEC4CEC5DE32C
:1050B000C501B4010E94C3364B015C010FC07720CB
:1050C00069F020E030E040E251E4C501B4010E9403
:1050D000C3364B015C017A9417149CF3662021F0CF
:1050E000B7FAB094B7F8B094F60180829182A282A8
:1050F000B382CE19DF09C150F801C08381E001C03D
:1051000080E0DF91CF911F910F91FF90EF90DF90A2
:10511000CF90BF90AF909F908F907F906F900895A9
:10512000009741F0EFE9FFE03197F1F700C0000090
:105130000197F6CF08958F929F92AF92BF92CF9230
:10514000DF92EF92FF9269017A019B01AC010E940C
:10515000C3364B015C01A7019601C701B6010E944D
:10516000C3369B01AC01C501B4010E94AC33FF9072
:10517000EF90DF90CF90BF90AF909F908F900C9466
:105180005037EBE6F0E08081897E8083E8E6F0E04E
:1051900080818E7F8083089584B1897E84B99091C7
:1051A000210785B196FF02C0897E01C0866185B95D
:1051B00093FF0BC080916B00866180936B008091A0
:1051C000680081608093680008950C94C1281F9244
:1051D0000F920FB60F9211242F933F934F935F932B
:1051E0006F937F938F939F93AF93BF93EF93FF93AF
:1051F00080919205813071F08091930585FD0AC000
:105200000E9418099FB7F894809193058066809357
:1052100093059FBFFF91EF91BF91AF919F918F91A8
:105220007F916F915F914F913F912F910F900FBEA2
:105230000F901F9018952F923F924F925F926F920E
:105240007F928F929F92AF92BF92CF92DF92EF9216
:10525000FF920F931F93CF93DF93CDB7DEB76C9779
:105260000FB6F894DEBF0FBECDBF898F8091910538
:105270008111CEC1409028075090290760902A07DD
:1052800070902B0708E017E0188F0F8B9E01235FAB
:105290003F4F59018E01005F1F4F212C1D8A812C29
:1052A000912C312C832D0E943F23D8018D938D01A9
:1052B000832D0E942B23F50181935F01AF89B88D67
:1052C000CD90DD90ED90FD90B88FAF8BA70196014A
:1052D000622D7D89C4010E94883618161CF0C22CEC
:1052E000DD8874013394B3E03B1621F02C2CDD8A69
:1052F0004701D8CF20E030E040EC5FEBC701B601BA
:105300000E94C3364B015C010E946424E6E0ED8BF1
:1053100033243394F98CEF2CF12CF88EEF8A95011D
:1053200084013058098F1A8F2B8F3C8F9E01205F8C
:105330003F4F3C8B2B8B8091210786FD02C0232C95
:1053400003C0222423942324A09123076A2F70E012
:10535000DE01119680E090E0D12C40E0582FEF89DB
:10536000F88D082E02C0F595E7950A94E2F79F01A3
:1053700021703327E0FF13C04F5F31100AC0E98C62
:10538000FA8C0B8D1C8DED92FD920D931C9313974F
:105390000BC08D929D92AD92BC92139705C01D9249
:1053A0001D921D921C921397FB0102C0F595E79583
:1053B0005A95E2F7E0FF0EC0ED90FD900D911C9123
:1053C000139717FB109517F91095ED92FD920D9319
:1053D0001C931397232B41F0EDE0F0E0EC0FFD1F41
:1053E000E80FF91F2081D22A019614968330910587
:1053F00009F0B4CF642F70E080E090E00E94253582
:105400000E9450379B01AC01D0929405C301B201B8
:105410000E94C336AB01BC01C12CE12CF12C8701E9
:1054200020E0CE0101960E94BB240E948C190E94AC
:105430005B1616E183B121108127DE015096FE0133
:105440003D962191922F9D2129F09C91982311F056
:105450002095D22211962B893C89E217F30789F710
:10546000D09294050E948C198091930584FF03C00B
:105470000E942715CDC08D2D8C71E1F60E941C195C
:105480000E94642480912C0790912D070E949028FF
:1054900040902407509025076090260770902707BA
:1054A00081E038263D8931503D8B311144CF8091C8
:1054B0002307E82EF12CFE8AED8AC0902E07D090AB
:1054C0002F07E0903007F0903107970186013058A0
:1054D000098F1A8F2B8F3C8F85E9A82E85E0B82E77
:1054E00094EE292E96E0392E9E012F5F3F4F490101
:1054F00000E010E08F89988D002E02C09595879569
:105500000A94E2F780FF3DC08D899E89002E02C07B
:10551000959587950A94E2F780FF23C0D101949670
:105520004D905D906D907C909797A3019201C7017B
:10553000B6010E94AC33F40160837183828393834C
:10554000D1012D913D914D915C91C301B2010E9419
:10555000C3360E949336F5016083718382839383FF
:1055600023C0898D9A8DAB8DBC8DF401808391838E
:10557000A283B383D5011D921D921D921C92139795
:1055800013C0F50160817181828193810E9427356A
:10559000D1012D913D914D915C910E948C34F4018B
:1055A00060837183828393830F5F1F4FF4E08F0EBC
:1055B000911C24E0A20EB11C34E0230E311C0330F8
:1055C000110509F097CF0E949C2740912807509120
:1055D000290760912A0770912B07C12CE12CF12C2F
:1055E000870120E0CE0101960E94BB2488E08093D1
:1055F00092059FB7F89480919305826080939305FC
:105600009FBF0E9427150E94411684E08093920557
:105610006C960FB6F894DEBF0FBECDBFDF91CF9171
:105620001F910F91FF90EF90DF90CF90BF90AF90C0
:105630009F908F907F906F905F904F903F902F90B2
:105640000895CF92DF92EF92FF920F931F93CF9323
:10565000DF938C01C8E0D7E0F801C190D190E190D0
:10566000F1908F0120E030E0A901C701B6010E944E
:105670008836181654F02991399149915991C701EA
:10568000B6010E94853487FF27C080919205803142
:1056900079F49FB7F894809193058860809393057F
:1056A0009FBF0E942715809191058823D1F319C0CF
:1056B0000E9418099FB7F8948091930580668093A3
:1056C00093059FBFDF91CF911F910F91FF90EF90B6
:1056D000DF90CF900C942715F7E0C431DF0709F075
:1056E000BBCFDF91CF911F910F91FF90EF90DF9093
:1056F000CF900895CF93DF93EC018991882319F01F
:105700000E947214FACFDF91CF910895CF93DF9367
:10571000FC018491EF012196882321F00E947214EC
:10572000FE01F7CFDF91CF910895EF92FF920F9393
:105730001F93CF93DF93CDB7DEB728970FB6F894BA
:10574000DEBF0FBECDBFFE0131967F019E01275FF8
:105750003F4F982F917091938695E217F307C9F701
:105760008F01F80182918F01805D0E9472140E15E5
:105770001F05B9F728960FB6F894DEBF0FBECDBF50
:10578000DF91CF911F910F91FF90EF9008951F939C
:10579000CF93DF9300D01F92CDB7DEB7811109C040
:1057A00080E30F900F900F90DF91CF911F910C9499
:1057B000721490E02AE011E0190FE1E0F0E0EC0F44
:1057C000FD1FE90FF11D622F0E94BB37905D908392
:1057D000882311F0912FEFCF112341F0FE01E10F4B
:1057E000F11D80810E9472141150F6CF0F900F901E
:1057F0000F90DF91CF911F9108958F929F92AF925A
:10580000BF92CF92DF92EF92FF920F931F93CF93AD
:10581000DF93CDB7DEB72A970FB6F894DEBF0FBE81
:10582000CDBF6B017C01142F20E030E0A9010E9464
:10583000853487FF07C08DE20E947214F7FAF09456
:10584000F7F8F094012F023060F020E030E048ECEF
:1058500052E4C701B6010E94C3366B017C010250BD
:10586000F2CF10FF0AC020E030E040E251E4C7016F
:10587000B6010E94C3366B017C0120E030E040E0BD
:105880005FE3C701B6010E94AC330E94F434E1E04B
:10589000F0E0EC0FFD1FE10FF11D2EE22083D12C73
:1058A0003AE0832E912CA12CB12C61157105810554
:1058B0009105A9F0D11201C0D394EE24E394F12C08
:1058C000EC0EFD1EED0CF11CA50194010E94C737E2
:1058D000605DF7016083B901CA01D394E6CF80E32C
:1058E000D11648F4E1E0F0E0EC0FFD1FED0DF11DE5
:1058F0008083D394F5CF8D2DD1120BC0D394D39444
:105900008F5FE1E0F0E0EC0FFD1FE80FF11D80E399
:105910008083DD2041F0FE01ED0DF11D80810E94AC
:105920007214DA94F6CF2A960FB6F894DEBF0FBE43
:10593000CDBFDF91CF911F910F91FF90EF90DF903E
:10594000CF90BF90AF909F908F90089520912107A6
:1059500020FF08C02BE832E441E25DE30E94C33639
:1059600044E001C043E00C94FD2B2091210720FF6F
:1059700008C02BE832E441E25DE30E94C33641E017
:1059800001C040E00C94FD2B43E00C94FD2B3D98AE
:105990008091210787FF04C045981092320708952F
:1059A000459A80E280933207089586B18072909183
:1059B0003207892708958091A2058130A1F40E94C1
:1059C000D52C882381F01092A2058CE0E5E9F5E062
:1059D000A3EAB5E001900D928A95E1F780919305D5
:1059E0008860809393050895CF93C82F811103C0D9
:1059F00088E598E044C080E598E00E94862B4C2F13
:105A000050E0FA013197E631F10580F5E658FF4F95
:105A10000C94E93788E398E002C086E298E00E949F
:105A2000862B2BC084E198E0FACF8AE098E0F7CF8C
:105A300089EF97E0F4CF8AEE97E0F1CF89EC97E019
:105A4000EECF80EC97E0EBCF85EB97E0E8CF82EAF2
:105A500097E0E5CF84E997E0E2CF8EE797E0DFCFEC
:105A60008AE697E0DCCF86E597E0D9CF84E497E03B
:105A70000E94862B8C2F0E94C72B81E497E0CF9148
:105A80000C94862BCF93C82F89E397E00E94862B36
:105A9000CE3F51F0CF3F29F0CD3F51F48BE097E05E
:105AA00005C089E297E002C086E197E00E94862B5C
:105AB00088E097E00E94862B84EF91E0CF910C94D0
:105AC0009028CF93C82F86E097E00E94862BC330A2
:105AD00091F038F4C13061F0C230A1F480EE96E06C
:105AE0000FC0C43059F0C53069F48DEB96E008C0A2
:105AF00084EF96E005C08EEC96E002C086EC96E05E
:105B00000E94862B89EB96E0CF910C94862B84E93A
:105B100096E00C94862B80E595E00C94862BFF9202
:105B20000F931F93CF93DF938CE495E00E94862B15
:105B3000809114070E94C72B83E395E00E94862B77
:105B4000809117070E94C72B85E195E00E94862B64
:105B5000809115070E94C72B8CEF94E00E94862B42
:105B6000809115070E94952B85EF94E00E94862B6B
:105B7000809116070E94C72B8DED94E00E94862B22
:105B8000809116070E94952B86ED94E00E94862B4B
:105B900080912107909122079695879596958795F4
:105BA00081700E94C72B85EB94E00E94862B809128
:105BB00021079091220736E0969587953A95E1F76F
:105BC00081700E94C72B85E994E00E94862B80910A
:105BD000210790912207880F892F881F990B919593
:105BE00081700E94C72B85E794E00E94862B8091EC
:105BF00018070E94C72B8FE594E00E94862B8091A6
:105C000018070E94952B87E594E00E94862B6091EF
:105C1000190770911A0780911B0790911C070E9429
:105C2000C42C87E394E00E94862B60911D0770913D
:105C30001E0780911F07909120070E94C42C8CE1C1
:105C400094E00E94862B8091210781700E94C72BCF
:105C50008FEF93E00E94862B80912107909122077D
:105C60009695879581700E94C72B85EE93E00E94E0
:105C7000862B809121079091220765E09695879564
:105C80006A95E1F781700E94C72B8AEC93E00E942D
:105C9000862B809121079091220773E09695879536
:105CA0007A95E1F781700E94C72B8FEA93E00E94FA
:105CB000862B8091210790912207E4E096958795A5
:105CC000EA95E1F781700E94C72B83E993E00E9477
:105CD000862B809123070E94C72B89E793E00E94BF
:105CE000862B809123070E94952B81E793E00E94E9
:105CF000862B60912407709125078091260790914B
:105D000027070E94C42C84E593E00E94862B6091B3
:105D100028077091290780912A0790912B070E94EC
:105D2000C42C87E393E00E94862B80912C070E946D
:105D3000C72B88E193E00E94862B60912E0770911B
:105D40002F0780913007909131070E94C42C8FEF6C
:105D500092E00E94862B8AEF92E00E94862B80912F
:105D6000220781700E94C72B8CED92E00E94862B47
:105D7000F4E6FF2E10E0C4EED6E000E08AED92E0FB
:105D80000E94862B802F8F0D0E94C72B88ED92E0FA
:105D90000E94862B123071F01330B9F0113029F0C7
:105DA000688179818A819B8117C06C857D858E850C
:105DB0009F8512C020E030E041E655E4688D798D82
:105DC0008A8D9B8D0E948C3407C08CA19DA1AEA1B1
:105DD000BFA1BC01CD0190580E94C42C85ED92E07A
:105DE0000E94862B013029F0023031F083ED92E0E1
:105DF00005C081ED92E002C08FEC92E00E94862BFC
:105E0000123051F0133059F0113019F085EC92E056
:105E100008C083EB92E005C082EA92E002C082E90A
:105E200092E00E94862B8EE892E00E94862B0F5F04
:105E30002496033009F0A2CF8AE0F80E1F5F8CE8A9
:105E4000F81299CFDF91CF911F910F91FF90089594
:105E5000CF92DF92FF920F931F93CF93DF9300D0E7
:105E600000D0CDB7DEB788E892E00E94862B03EA27
:105E700015E084EEC82E86E0D82EF12CF801619151
:105E80007191819191918F01F6012191319141910F
:105E900051916F0129833A834B835C830E9427359C
:105EA00029813A814B815C810E948C340E94A62C0E
:105EB000F2E0FF1621F086E892E00E94862BF39430
:105EC00083E0F812DBCF82E892E00F900F900F9002
:105ED0000F90DF91CF911F910F91FF90DF90CF90A6
:105EE0000C94862BEF92FF920F931F93CF93DF9327
:105EF000CDB7DEB72C970FB6F894DEBF0FBECDBF7F
:105F0000F12CBE016F5F7F4F8F2D0E949C2181116C
:105F100004C087E00E94F42C69C08FE792E00E94E1
:105F2000862B86E0F81631F0E7E0FE1208C089E71C
:105F300092E002C08CE792E00E94862B04C086E3C8
:105F40008F0D0E94C72B87E792E00E94862B8E015F
:105F50000F5F1F4FE12CF801619171918191919137
:105F60008F010E94A62CF2E0EF1619F085E792E06F
:105F700002C081E792E00E94862BE39483E0E8125E
:105F8000EACFF394E8E0FE12BCCF8BE692E00E94E9
:105F9000862B0AED15E0F12CF80161917191819148
:105FA00091918F010E94A62CF2E0FF1619F089E66C
:105FB00092E002C085E692E00E94862BF39483E093
:105FC000F812EACF8FE592E00E94862B6091E605F9
:105FD0007091E7058091E8059091E9050E94A62C53
:105FE0008BE592E00E94862B0E94282F2C960FB6FC
:105FF000F894DEBF0FBECDBFDF91CF911F910F91FF
:10600000FF90EF9008958091AF05823091F038F4C1
:10601000882361F08130A1F483E592E00FC08330E2
:1060200059F0853069F486E492E008C087E592E093
:1060300005C08FE492E002C08BE492E00E94862BC0
:1060400083E492E00E94862B8091B5058A5C0E94D1
:10605000C72B8091B305813049F028F0823051F48C
:1060600084E392E005C08EE392E002C089E392E00F
:106070000E94862B8091B105811103C08FE292E0CE
:1060800002C08AE292E00E94862B8091B2058111C3
:1060900003C085E292E002C080E292E00E94862B7B
:1060A0008091B005813019F48BE192E002C086E165
:1060B00092E00E94862B8091B605813049F028F04D
:1060C000823051F48AE092E005C082E192E002C0A1
:1060D0008EE092E00E94862B8091B805813031F0ED
:1060E00040F0823051F482E092E005C086E092E018
:1060F00002C08EEF91E00E94862B8091B705882325
:1061000029F0823039F486EF91E002C08AEF91E005
:106110000E94862B83EF91E00E94862B8091C1051F
:106120000E94C72B80EF91E00E94862B6091BD05F5
:106130007091BE058091BF059091C0050E94B52C5D
:106140008DEE91E00E94862B6091B9057091BA05A1
:106150008091BB059091BC050E94B52C89EE91E021
:106160000C94862B1F93CF93DF93182FEB0186EEB1
:1061700091E00E94862B812F0E94C72B84EE91E034
:106180000E94862BCE010E947A2B81EE91E0DF9156
:10619000CF911F910C94862BCF93DF93EC0182ED6E
:1061A00091E00E94862BCE010E947A2B8EEC91E02A
:1061B000DF91CF910C94862BBF92CF92DF92EF921A
:1061C000FF920F931F93CF93DF93CDB7DEB76C97FA
:1061D0000FB6F894DEBF0FBECDBF8CE0E5E9F5E069
:1061E000DE011D9601900D928A95E1F7809192054E
:1061F0008430D9F040F48130D9F070F08230E1F48D
:1062000082EA91E017C0803151F0803259F0883035
:1062100099F481EC91E00EC088EC91E00BC08CEB1E
:1062200091E008C086EB91E005C080EB91E002C0F0
:1062300089EA91E00E94862B8091180780FD05C0B5
:106240008091180781FF8AC03CC08BE991E00E94D1
:10625000862B6E012DE0C20ED11C94EEE92E96E045
:10626000F92E8E010F5F1F4FB12CF60161917191D4
:10627000819191916F01F70121913191419151915A
:106280007F01298F3A8F4B8F5C8F0E942735298D94
:106290003A8D4B8D5C8D0E948C34F8016193719323
:1062A000819391938F010E94A62CF2E0BF1621F0FA
:1062B00089E991E00E94862BB39423E0B212D5CFF6
:1062C000BFCF82E991E00E94862B8EECE82E85E01C
:1062D000F82E8E010F5F1F4FB12C6801F7016191FD
:1062E0007191819191917F012085318542855385FE
:1062F0000E94AC339B01AC01F80160817181828105
:1063000093810E94AB33F80160837183828393830E
:10631000F2E0BF120FC02091E6053091E7054091F1
:10632000E8055091E9050E94AB33F8016083718361
:10633000828393830C5F1F4FF6016081718182819C
:1063400093810E94A62CF2E0BF1621F080E991E033
:106350000E94862BB39423E0B212BFCF8CE891E069
:106360000E94862B8091B3000E94C72B8091180752
:1063700082FF08C086E891E00E94862B0E94CD270C
:106380000E94C72B8091180783FF08C081E891E025
:106390000E94862B0E9453140E94C72B89E791E02C
:1063A0000E94862B8091B00087FF03C085E791E0B3
:1063B00002C080E791E00E94862B8091B3000E948A
:1063C000C72B8CE691E06C960FB6F894DEBF0FBE3B
:1063D000CDBFDF91CF911F910F91FF90EF90DF9094
:1063E000CF90BF900C94862B87B1887F87B988B1F6
:1063F000876088B9ECE6F0E0808187608083E8E61A
:10640000F0E080818260808308951F920F920FB622
:106410000F9211242F933F934F935F936F937F932A
:106420008F939F93AF93BF93EF93FF9386B190E0C9
:106430008095909587709927892B91F0309903C0AA
:106440000E9418090DC0319904C08091930588609D
:1064500005C0329905C080919305826080939305B1
:10646000FF91EF91BF91AF919F918F917F916F912C
:106470005F914F913F912F910F900FBE0F901F9002
:1064800018951F93CF93DF93EC0110E0BE01812F8D
:106490000E946C21811102C087E009C08881882395
:1064A00041F0CE010E947A2BCE010E94BD090E94CC
:1064B000F42C1F5F123051F7DF91CF911F91089597
:1064C0008F929F92AF92BF92CF92DF92EF92FF9204
:1064D0001F93CF93DF93CDB7DEB729970FB6F8940C
:1064E000DEBF0FBECDBF7C0181E08987F7018181CE
:1064F000833419F12CF4882341F0843249F045C0EB
:10650000873491F0883589F140C00E948B2D0AC0F4
:1065100082E08987F7018281882311F083E009C135
:106520000E948F2D80E005C182E08987F70182817A
:106530008111F4CF0E940330F5CF82E08987F70103
:1065400092819111EBCF90919205923021F40E94AB
:10655000180985E007C0992311F088E0EAC080930C
:10656000920584E00E94612DDDCF82E08987F701EA
:1065700082818111D3CF80919205813099F683E099
:106580000E94612D10929205CDCF9091920592308C
:1065900020F7883491F01CF4833231F05BC08934E9
:1065A000D1F08E34C9F156C082E08987F70182812B
:1065B0008111B4CF0E94722FB5CF8091210784FF43
:1065C000B7C00E943709809191058111ABCFC701F7
:1065D0000E944132A7CF82E08987F7018281811131
:1065E00007C0C7010E948921C7010E94CC309ACF01
:1065F0008D3309F093CF83E0F701E80FF11D90810F
:10660000DF0113979C938F5F90819111F5CF89875C
:10661000C7010E94792086CF82E08987F7018281B5
:10662000811114C010E0B701812F0E946C218111EB
:1066300004C087E00E94F42C04C0B701812F0E949F
:10664000B2301F5F123009F46DCFEDCF911185CFBD
:1066500011E001C010E0AE014B5F5F4FBE01675F0C
:106660007F4FC7010E94DE27811102C082E061C016
:10667000898521E0280F2987F701E80FF11D808126
:106680008D3309F04BCF112321F1822F90E0E22FBF
:10669000F0E0D701AE0FBF1F3C91E81BF90BEE0DE8
:1066A000FF1D30832F5F3C913111F1CF2987C70146
:1066B0000E94BD0981113DC06D817E818F819885C9
:1066C0000E9491370E94F934862FB7010E947020F2
:1066D00029CFAE014F5F5F4FBE01675F7F4FC7019C
:1066E0000E94DE27882311F28985F701E80FF11D4A
:1066F0008081811113CFCD80DE80EF80F88420E08F
:1067000030E04FE753E4C701B6010E9488361816FF
:106710000CF404CF89809A80AB80BC80C701B6019D
:106720000E94F934862FB501A4010E94D12101C035
:1067300085E029960FB6F894DEBF0FBECDBFDF917E
:10674000CF911F91FF90EF90DF90CF90BF90AF90CF
:106750009F908F9008955058BB27AA270ED076C2DD
:106760003FD230F044D220F031F49F3F11F41EF4B8
:106770000FC20EF4E095E7FBDCC1E92F89D280F36C
:10678000BA17620773078407950718F071F49EF52E
:10679000B8C20EF4E0950B2EBA2FA02D0B01B90153
:1067A00090010C01CA01A0011124FF27591B99F087
:1067B000593F50F4503E68F11A16F040A22F232F93
:1067C000342F4427585FF3CF469537952795A795E3
:1067D000F0405395C9F77EF41F16BA0B620B730B8A
:1067E000840BBAF09150A1F0FF0FBB1F661F771FFB
:1067F000881FC2F70EC0BA0F621F731F841F48F4B0
:10680000879577956795B795F7959E3F08F0B3CF35
:106810009395880F08F09927EE0F9795879508951F
:10682000DFD158F080E891E009F49EEFE0D128F044
:1068300040E851E059F45EEF09C0AAC162C2E92FF5
:10684000E07826D268F3092E052AC1F32617370708
:106850004807590738F00E2E07F8E02569F0E025C3
:10686000E0640AC0EF6307F8009407FADB01B9019E
:106870009D01DC01CA01AD01EF935DD0E7D10AD0E3
:106880005F91552331F02BED3FE049E450FD49EC99
:1068900063CF0895DF93DD27B92FBF7740E85FE32B
:1068A0001616170648075B0710F4D92F35D29F93A9
:1068B0008F937F936F9332D3E0E2F1E06CD1C6D136
:1068C0002F913F914F915F916AD2DD2349F090580B
:1068D000A2EA2AED3FE049EC5FE3D0785D274DDF87
:1068E000DF91B4C1F7D180F09F3740F491110EF4DD
:1068F00009C260E070E080E89FE3089526F01B166F
:10690000611D711D811D1BC135C1EFD008F481E0EF
:10691000089575D1E395ABC10CD098C168D140F012
:106920005FD130F021F45F3F19F003C15111EAC18A
:106930002FC1AED198F39923C9F35523B1F3951B19
:10694000550BBB27AA2762177307840738F09F5F90
:106950005F4F220F331F441FAA1FA9F333D00E2EFF
:106960003AF0E0E830D091505040E695001CCAF76C
:1069700029D0FE2F27D0660F771F881FBB1F261731
:1069800037074807AB07B0E809F0BB0B802DBF0104
:10699000FF2793585F4F2AF09E3F510568F0C9C00A
:1069A000B1C15F3FECF3983EDCF386957795679530
:1069B000B795F7959F5FC9F7880F911D96958795B5
:1069C00097F90895E1E0660F771F881FBB1F6217D4
:1069D00073078407BA0720F0621B730B840BBA0B92
:1069E000EE1F88F7E095089504D06894B1118AC12C
:1069F000089556D188F09F5790F0B92F9927B75135
:106A0000A0F0D1F0660F771F881F991F1AF0BA9572
:106A1000C9F712C0B13081F074D1B1E0089571C1ED
:106A2000672F782F8827B85F39F0B93FCCF3869568
:106A300077956795B395D9F73EF4909580957095C5
:106A400061957F4F8F4F9F4F0895E89409C097FB42
:106A50003EF490958095709561957F4F8F4F9F4F35
:106A60009923A9F0F92F96E9BB279395F695879579
:106A700077956795B795F111F8CFFAF4BB0F11F43C
:106A800060FF1BC06F5F7F4F8F4F9F4F16C08823E3
:106A900011F096E911C0772321F09EE8872F762F19
:106AA00005C0662371F096E8862F70E060E02AF05A
:106AB0009A95660F771F881FDAF7880F9695879546
:106AC00097F9089507D180F09F3740F491110EF0A7
:106AD00019C160E070E080E89FEB089526F41B1672
:106AE000611D711D811D2BC045C0990F0008550FF8
:106AF000AA0BE0E8FEEF16161706E807F907C0F044
:106B000012161306E407F50798F0621B730B840B4B
:106B1000950B39F40A2661F0232B242B252B21F425
:106B200008950A2609F4A140A6958FEF811D811DC5
:106B3000089597F99F6780E870E060E008958823E2
:106B400071F4772321F09850872B762F07C06623A6
:106B500011F499270DC09051862B70E060E02AF067
:106B60009A95660F771F881FDAF7880F9695879595
:106B700097F908959F3F31F0915020F487957795CC
:106B80006795B795880F911D9695879597F9089504
:106B90009FEF80EC0895DF93CF931F930F93FF92A5
:106BA000EF92DF927B018C01689405C0DA2EEF0131
:106BB000F6D0FE01E894A591259135914591559126
:106BC000AEF3EF01DADDFE019701A801DA9479F75F
:106BD000DF90EF90FF900F911F91CF91DF9108957B
:106BE00000240A94161617061806090608950024AC
:106BF0000A9412161306140605060895C9CF50D03C
:106C0000E8F3E894E0E0BB279F57F0F02AED3FE07F
:106C100049EC06C0EE0FBB0F661F771F881F28F0D8
:106C2000B23A62077307840728F0B25A620B730BFB
:106C3000840BE3959A9572F7803830F49A95BB0FE0
:106C4000661F771F881FD2F7904896CF092E0394AE
:106C5000000C11F4882352F0BB0F40F4BF2B11F449
:106C600060FF04C06F5F7F4F8F4F9F4F0895EF937A
:106C7000E0FF06C0A2EA2AED3FE049EC5FEB7DDDD4
:106C8000E5DF0F90039401FC9058EDE4F1E057C16B
:106C900057FD9058440F551F59F05F3F71F04795CD
:106CA000880F97FB991F61F09F3F79F087950895B2
:106CB000121613061406551FF2CF4695F1DF08C0D1
:106CC000161617061806991FF1CF869571056105EE
:106CD00008940895E5DFA0F0BEE7B91788F4BB2754
:106CE0009F3860F41616B11D672F782F8827985F9C
:106CF000F7CF869577956795B11D93959639C8F32B
:106D00000895E894BB2766277727CB0197F9089564
:106D1000ECDE08F48FEF08959B01AC0160E070E0B9
:106D200080E89FE3F9CDBCDF58F19E5758F19851A8
:106D3000A0F0E9F0983020F5092E9927660F771F0B
:106D4000881F991F0A94D1F712C0062E672F782F3B
:106D50008827985F11F4000C07C0993FB4F386951B
:106D6000779567959395D9F7611D711D811D3EF447
:106D700090958095709561957F4F8F4F9F4F0895A7
:106D80006894C0CFBECF0BD061CF2ADF28F02FDFB1
:106D900018F0952309F0CDCEFBCE1124B3CF78DFC8
:106DA000A0F3959FD1F3950F50E0551F629FF0011E
:106DB000729FBB27F00DB11D639FAA27F00DB11D77
:106DC000AA1F649F6627B00DA11D661F829F222700
:106DD000B00DA11D621F739FB00DA11D621F839F87
:106DE000A00D611D221F749F3327A00D611D231F5D
:106DF000849F600D211D822F762F6A2F11249F57AB
:106E000050408AF0E1F088234AF0EE0FFF1FBB1FCD
:106E1000661F771F881F91505040A9F79E3F51056C
:106E200070F087CE6FCF5F3FECF3983EDCF3869532
:106E300077956795B795F795E7959F5FC1F7FE2B17
:106E4000880F911D9695879597F9089529DFE0F0B1
:106E50009E37D8F09639B8F49E3848F4672F782FCB
:106E60008827985FF9CF869577956795939595399B
:106E7000D0F3B62FB1706B0F711D811D20F4879573
:106E80007795679593955BCE75CE3CCF9F93B7DE94
:106E90000F9007FCEE5FEBCE11F40EF479CE6ACEC4
:106EA000FFDED0F39923D9F3CEF39F57550B87FF1D
:106EB0003FD00024A0E640EA90018058569597956F
:106EC00028F4805C660F771F881F20F0261737078D
:106ED000480730F4621B730B840B202931294A2B9D
:106EE000A69517940794202531254A2758F7660F51
:106EF000771F881F20F026173707480730F4620BEA
:106F0000730B840B200D311D411DA09581F7B90134
:106F1000842F9158880F9695879508959B01AC0111
:106F200032CFD8DE20F09F3708F4ECCE08CE22CE48
:106F300091505040660F771F881FD2F708959F9396
:106F40008F937F936F93FF93EF939B01AC011BDFB4
:106F5000EF91FF9120DE2F913F914F915F9113CFE1
:106F60000E94EF37A59F900DB49F900DA49F800DB8
:106F7000911D11240895991B79E004C0991F96175B
:106F800008F0961B881F7A95C9F780950895A1E2AD
:106F90001A2EAA1BBB1BFD010DC0AA1FBB1FEE1F93
:106FA000FF1FA217B307E407F50720F0A21BB30BDE
:106FB000E40BF50B661F771F881F991F1A9469F75A
:106FC00060957095809590959B01AC01BD01CF01B6
:106FD0000895EE0FFF1F0590F491E02D0994A29FF4
:106FE000B001B39FC001A39F700D811D1124911D9D
:106FF000B29F700D811D1124911D0895F894FFCF4B
:0670000000003307200030
:00000001FF
